:020000040000FA
:1000000040130820D9010000E1010000E3010000D5
:10001000E5010000E7010000E90100000000000028
:10002000000000000000000000000000EB010000E4
:10003000ED01000000000000EF010000F1010000F0
:10004000F3010000ED090000E54F000073500000CF
:1000500059080000F3010000F3010000F301000063
:10006000F3010000F3010000F3010000F3010000C0
:10007000F3010000F3010000F3010000F3010000B0
:10008000F3010000F3010000F3010000F3010000A0
:10009000F301000037080000F3010000F301000045
:1000A000F3010000F3010000F3010000F301000080
:1000B000F3010000F3010000F3010000CD07000090
:1000C000F301000000F002F800F05CF80AA090E8EC
:1000D000000C82448344AAF10107DA4501D100F003
:1000E00051F8AFF2090EBAE80F0013F0010F18BF74
:1000F000FB1A43F001031847008100003081000023
:100100000A444FF0000C10F8013B13F0070408BF3D
:1001100010F8014B1D1108BF10F8015B641E05D0DB
:1001200010F8016B641E01F8016BF9D113F0080F90
:100130001EBF10F8014BAD1C0C1B09D16D1E58BF22
:1001400001F801CBFAD505E014F8016B01F8016B59
:100150006D1EF9D59142D6D37047000000230024CC
:1001600000250026103A28BF78C1FBD8520728BFC7
:1001700030C148BF0B6070471FB506F054FB1FBD70
:1001800010B510BD06F05CFC1146FFF7F5FF02F05C
:10019000E2FA06F07AFC03B4FFF7F2FF03BC06F0C4
:1001A0007BFC00000B49D1F800C04A685CF8043BB6
:1001B0001068184442F8040B8C4528BFA1F1DC0CF0
:1001C0008A4228BFA1F1DC02C1F800C04A6020F0D9
:1001D0000040704734F3072009488047094800472A
:1001E000FEE7FEE7FEE7FEE7FEE7FEE7FEE7FEE7E7
:1001F000FEE7FEE704480549034A054B7047000047
:1002000047030000C50000004053001040130820C1
:1002100040F3072095480068C0F30160032860D1CF
:1002200092488430006800F0030030B1012820D0EB
:10023000022839D0032853D100E000BF8B48006862
:10024000C0F30E00401C4000894948438749883963
:10025000D1F88810C1F30741491CB0FBF1F1834884
:100260007C300068C0B2401CB1FBF0F081490860EE
:1002700036E07E480068C0F30E00401C40007E4916
:1002800048437A498839D1F88810C1F30741491C9D
:10029000B0FBF1F175487C300068C0B2401CB1FB86
:1002A000F0F0744908601BE070480068C0F30E006D
:1002B000401C40004FF4FA4148436C498839D1F85A
:1002C0008810C1F30741491CB0FBF1F167487C304D
:1002D0000068C0B2401CB1FBF0F06649086000BF86
:1002E00030E062488430006800F0030030B101283B
:1002F00010D0022819D0032823D100E000BF5B48AA
:100300007C300068C0B2401C5949B1FBF0F059493B
:10031000086016E055487C300068C0B2401C564961
:10032000B1FBF0F0534908600BE050487C300068A6
:10033000C0B2401C4FF4FA41B1FBF0F04D490860E7
:1003400000BF00BF704720204C49086000BF4B48E9
:10035000006800F040000028F9D0032043497C31B8
:100360000860012041498839C1F80C0144483F49DF
:10037000091F0860AA203D49091D08605520086032
:1003800001203A4908390860AA203849091D086047
:10039000552036498839C1F88C0000BF33480068C1
:1003A00000F080600028F9D0032030490839086047
:1003B000AA202E498839C1F88C0055202B49091DE7
:1003C000086000BF2948006800F040700028F9D09C
:1003D000232026491C310860AA2024498839C1F805
:1003E000AC00552021492431086001201F491831F3
:1003F0000860AA201D492431086055201B4988390E
:10040000C1F8AC0000BF19482030006800F48060DB
:100410000028F8D00320154918310860AA20134994
:100420008839C1F8AC00552010492431086000BF5C
:100430000E482030006800F440700028F8D01020EA
:100440000E4908310860002008498839C1F8AC011C
:100450000C4806493C3108600020084928310860F2
:1004600043F23A00014988390860704788C00F405C
:1004700000093D0000C00720001BB700A0C10F40CD
:1004800063000500DE8768042820A54908614FF451
:10049000BE70486140F2C110C860084680890004FF
:1004A0008860142088620A20C8629E48C86143F2AE
:1004B000C8200862002070479B480068102815D3A8
:1004C0009748006B9949096888420AD29448406B62
:1004D00096490968884204D94FF080509449C8630E
:1004E00019E04FF080509249886314E08C48006B0B
:1004F0008E49096888420AD28948406B8B4909684D
:10050000884204D94FF000708949C86303E04FF076
:10051000007087498863704710B5002485480068DB
:100520008549096888426CDB8448006808BB7C48C0
:10053000806A5A2802D95A207949886278488068A6
:10054000000C7F49B1FBF0F0441E7548806AC0F191
:10055000640060434FF4C871B0FBF1F07049086368
:100560000846006BC0EB54004863012073490860E3
:1005700029E06B48806A6A49C96A08445A2805D943
:100580006748C06AC0F15A0065498862644880685B
:10059000000C6B49B1FBF0F0441E6148806AC0F169
:1005A00064005F49C96A084460434FF4C871B0FBF6
:1005B000F1F05B4908630846006BC0EB54004863E8
:1005C00000205E4908600A20554988631E20C863E0
:1005D0005C48006806F012F9FFF7E4FD5049C96B6A
:1005E000B0FBF1F201FB12004D49896B08444C4904
:1005F00048620846406A5049086000204D4908603A
:1006000004E04C480068401C4A49086010BD10B521
:100610004D484E49096850F821004D490968884203
:1006200006D949484949096850F8210048490860F5
:100630003D48006820B10A281AD010286DD138E052
:10064000FFF76AFF36488068C00A4249B1FBF0F004
:1006500041498861324880684049B1FBF0F00003AD
:100660003F49486604F084FC00203049086054E0AB
:100670002B48C16936480068A0F58030A0F5967017
:10068000A1EB80002649C8610846C0693549884207
:1006900002D935482249C8612148C069000C204967
:1006A000886200202A4908601D48806A2F49086036
:1006B00033E004F064FC00201C490860001F2C4952
:1006C000086000202B49086016E0204800780C38AC
:1006D000284909780844C0B21B4951F82000B0F5F8
:1006E000803F04D322480068401C2149086021480B
:1006F0000068401C1F4908601E4800680828E4DBA9
:10070000074880681A49096801EB4102C2EBC11130
:10071000A0EBC1000249886000BF00BF10BD00000F
:1007200034C40720F6FF090090C2072084C20720C6
:1007300000C0092014C0072018C007200CC00720E3
:10074000A086010078C207205815001094C2072027
:100750008CC2072000E1F50500800040000053072F
:10076000A0D10720A0252600804F120010C007202E
:100770001CC0072020C00720FA4800686FF0004125
:1007800088421FD00120F8490860F8480068E0B1AD
:10079000F748006818B10020F549086015E0F548F1
:1007A0008068F049096888420FD9F3480068F34926
:1007B0000968884209D10020EB4908600120EC4912
:1007C000086002E00020E84908607047EC48C06813
:1007D000EC490860EC48006800F0080068B10420AB
:1007E000EA490860EA480068401CE949086000F0EE
:1007F000010010B10C20E549086041F6FF70E249A4
:100800000831086070470221E24A516018B1810046
:10081000916101215160704741F6FF71DA4A083257
:10082000116018B1D84A083A116003E00821D64A8D
:10083000121F11607047CF488068CA4908600120C4
:100840004FF040214860D448006840F40060D2492D
:100850008C39C1F88C007047C6488068C14908606F
:100860000120CC490860C5480068C349086070474A
:1008700010B50020FFF7C7FF0120C6490860C64831
:10088000001D006820F40060C3498C39C1F8900055
:100890000846D0F88C0040F40060BF490860022090
:1008A0004FF0402148603F200860BC48006800F4D9
:1008B000003008B1002010BDB848006820F00100E9
:1008C000B749C1F830010846D0F8500120F00100C6
:1008D000C1F850018800406900F0400008B90020CC
:1008E000E9E7B048806840F00400AE4988603F20E6
:1008F0004FF040210860AC480068032804DD0A205E
:1009000088613220C86106E00A204FF040218861EA
:1009100041F28830C861A549097801F0300001F042
:1009200020FEA1480068022803D14CF25030FFF7A6
:100930006AFF0120BFE79E4800689E490968401A87
:100940009B490860084600689A490968B0EB610F46
:1009500007DA99489649086098480068401C97490A
:10096000086096480068032808D194480068401C35
:10097000924908604FF6FF70914908607F4800680F
:10098000401C7E4908607B4880698A49086070473E
:10099000AA204107886055208860704710B504463A
:1009A0008848006820F440508749C1F8A8010846EB
:1009B000D0F8A80140F480508249086002206D49B7
:1009C0004860032048610120886242F21070794932
:1009D000086008460068674988614815C8640120B6
:1009E00008650920486000F0F7F810BD4FF040217D
:1009F0000868096841F003014FF04022116000F0DF
:100A0000010171B17149896D41F040016F4A9165F1
:100A10004FF04021096841F001014FF04022116080
:100A2000704700F0020171B16849C96D41F04001A1
:100A3000664AD1654FF04021096841F002014FF04C
:100A400040221160ECE700F0040101B1E8E700BFCB
:100A5000E6E710B55E48006920F040605C49086137
:100A60000846006820F4400008605848006820F4F8
:100A70000060564908604848001D006820F4006086
:100A800045498C39C1F890000846D0F88C0040F4F4
:100A90000060C1F88C00152000F058F84A48D0F8E2
:100AA000A80120F00C004849C1F8A8010846D0F878
:100AB000A80140F00C004349086000204FF040219D
:100AC000C8603F20086039204861002088620867BC
:100AD0000A20886141F28830C861012000F07CF86A
:100AE00010BD10B53848C430006840F400003649E5
:100AF000C1F8C4000846D0F8AC0120F44040C1F869
:100B0000AC010846D0F8AC0140F480402D49091DE5
:100B1000086000201F49C860012008600320486168
:100B200001208862042000F011F810BD10B50020EB
:100B300000F052F827484FF08041486001200860DB
:100B4000AA20886055208860012010BD00F01F0297
:100B5000012191404209920002F1E022C2F8001105
:100B600070470000200000101C00001088C1072002
:100B70004400001000800140180000100000001028
:100B800000C00B4018C20720E0CF0B402800001027
:100B900048000010004009408C8002403041005065
:100BA000004000500000014094C1072080C1072090
:100BB000080000101400001000E1F505040000100A
:100BC00084C10720A8C10F4000C00F4000C0092009
:100BD00000C00240FFFF3F0000F01F0201219140D2
:100BE000024A430942F823107047000080E100E008
:100BF000F748C07800F0800018B10120F54908607E
:100C000002E00020F3490860F34800684FF6CF7116
:100C10000840F1490860EE48C078302101EA6000E0
:100C2000EE490860EC48006809680843EA49086032
:100C300070470020EA4908600220EA490860EA4853
:100C4000EA490860E64848600420E9490860012054
:100C50004860E849086070470120E74908600020C3
:100C6000DF4908600520DF490860DF482830DF4998
:100C70000860E2484860E2488860DB487038C86035
:100C8000803008610820DA490860042048600220AA
:100C90008860C8600C2008610120D6490860704750
:100CA000D848007800F0010090B9D64800684008A4
:100CB000D54951F82000D549086008460068006809
:100CC000D349086008460068000AD249086003E07A
:100CD000CF480068CF490860CE480078CD49086009
:100CE00008460068C749096840EA0120C949086008
:100CF0000020BB4908600220BA490860BA48001FBA
:100D0000BA490860C34848600220B9490860486091
:100D10000120B8490860BB480068401CB949086018
:100D200008460068152801D9002008607047012096
:100D3000AC490860B848AD490860B8480068400050
:100D4000AB49086008460068402801D3402008608D
:100D50000020A24908609F4908600120A549086059
:100D60007047AF48008800F47F40AD49086001201B
:100D70009C490860AA489D49086002209C49086077
:100D800001209C4908607047022096490860A548E8
:100D9000964908609048486002209549086048607C
:100DA00000208C490860012092490860704700B516
:100DB0009D48006850B38748006810B101208D49F4
:100DC00008609A480068012802D005281DD102E079
:100DD000FFF766FF19E0924800684FF61F71084060
:100DE0008F490860084600684DF6025188420BD1D1
:100DF0008F48006800F0080018B101207D490860A4
:100E000002E000207B49086000BF00BF00BD00B5C4
:100E10006F48C0788349086000206E490860FFF77A
:100E2000B3FF00BD00B56A48C07800F00F00684904
:100E3000C97820EA1112012A1CD101207D490860DD
:100E40006348007900067C49086061484079096878
:100E500041EA0040784908605D488079096841EAC4
:100E60000020754908605A48C079096808437249EA
:100E7000086002E000206F490860002055490860C2
:100E8000FFF782FF00BD00B504206C49086064488C
:100E9000007800F007024E4840794D49097940EA50
:100EA0000120A0F500405049703941F822005C480B
:100EB000007800F0800000B900BDFFF752FF00BFCE
:100EC000FAE700B5FFF794FE0220464908605C4847
:100ED000464908605B484860022045490860486010
:100EE00000203E4908603B490860012041490860F4
:100EF00000BD002054490860704700B5FFF731FF7E
:100F000000BD704710B5FFF773FE3448006801F06C
:100F100028FB0420334908600020344908604860F9
:100F200088604A48C860022031490860486088608B
:100F3000C86001202F49086010BD10B5FFF758FEAA
:100F40002648006801F00DFB02202649086026486B
:100F5000083026490860001D4860022024490860C6
:100F6000486001202349086010BD02201D49086027
:100F70002B481E49086002201D490860486014483B
:100F8000C07800F0100018B931481849486002E0F4
:100F9000194816494860224800684FF61071084009
:100FA0001F490860012013490860704702220D4B59
:100FB0001A601B4A0D4B1A6002220D4B1A605A60D0
:100FC000174A127802F010020AB9214843E041E0C2
:100FD000E4C407200C00001080C10720ECC00720EB
:100FE0008CC10720F0C0072010D2072064C507205D
:100FF000A4C50720F4C0072088C1072034000010D2
:101000003C00001070C0072038C007206CC00720CB
:1010100064C0072068C00720A4C40720E4C00720DC
:1010200028C0072094C107201C00001024C00720FE
:1010300028000010E0C10720DCC1072034C00720D1
:1010400030C0072090C10720F8C0072098D10720A2
:1010500084C10720F748F84A5060F84A127802F035
:101060000F01F64A127802F080022AB901238B4060
:1010700002689A43026004E001228A400368134335
:101080000360EE4A12684FF610731A40EB4B1A6079
:101090000022EB4B1A600122EA4B1A6070470120D4
:1010A000E9490860E948E44908600220E849086025
:1010B0000120E4490860704710B50120E549086047
:1010C000E5480179407961F31F20E4494866E24828
:1010D0008179C07961F31F20E049086600F03CFB8C
:1010E0000020D7490860FFF73CFE10BD10B5DA4874
:1010F0000079DB49C1F8E000D7484079C1F8E40045
:101100000A46D2F8E410D2F8E00003F0DBF9002040
:10111000CB490860FFF725FE10BD10B5FFF768FD4D
:10112000D048006801F01DFACB48C07800F01F04D9
:10113000082C46D2DFE804F0AC04465F74ACAC8DFA
:101140000020BC490860FFF767FBC748C749086033
:101150000E20BD4908600020C5490860BF487830AE
:10116000B5490860001D4860083888601838C860B4
:1011700050380861001D486154308861001DC86105
:1011800008380862BB484862B44888620830C862C0
:10119000783008632C3848630220AD490860486005
:1011A0008860C860086148618861C86108624862F7
:1011B0008862C862042048630C2008630120A149AA
:1011C000086065E000209B490860FFF725FB0020D0
:1011D000A649086002209C490860A04878309649DA
:1011E0000860001D4860022099490860486001209D
:1011F000944908604CE040F6C4109C490860022005
:1012000091490860954854308B490860001D48603A
:1012100002208F490860486001208A49086037E051
:1012200044F62060914908600420874908608B4893
:101230000C30814988600C38C860102084490860EF
:101240002020486002208860C86001207D49086035
:101250001EE044F620608549086005207A49086050
:101260007E48143074490860203048603438886003
:101270000830C860001D086110207549086048608A
:1012800002208860C860086101206E49086000BFC4
:1012900000BF76480068FFF7B6FA10BD00BFFEE752
:1012A0000120694908606C48C0786D4901EB8000F5
:1012B00061490860022066490860012061490860B0
:1012C000704700B5002063490860654A6248C078ED
:1012D00002EB800260480179407961F31F201060C1
:1012E000002057490860FFF73CFD00BD10B5032002
:1012F00003F0C7FB5A4890F8F0005F4908600020EF
:101300004F490860FFF72DFD10BD00B500204C4986
:101310000860FFF726FD00BD00B5012057490860B1
:10132000002047490860FFF71CFD00BD00B5012003
:1013300053490860002042490860FFF712FD00BDD4
:1013400000B501204F49086000203D490860FFF7C3
:1013500008FD00BD70477047704710B501204A492D
:1013600008603D48807804023B48C07820433349F8
:10137000086014B9FFF7EEFF10BDB4F5254F05D195
:10138000032042490860FFF742FDF5E7B4F5304F0E
:101390000ED1012027490860FFF72AFC3148006878
:1013A00001F0DFF8042039490860FFF742FCE3E769
:1013B000B4F5204F14D1FFF71BFC2A48006801F058
:1013C000D0F833480068042803DA02203049086066
:1013D00002E004202E49086001202C490860CBE778
:1013E000B4F5324F13D1FFF703FC072027490860FB
:1013F0001948C07800F0010018B1002025490860A4
:1014000002E0012023490860FFF726FCB4E7B4F5A9
:10141000274F05D106201D490860FFF703FDABE704
:10142000B4F5706F38D1022018490860FFF793FFB8
:10143000A2E7000088C1072064C5072028C0072054
:101440000C000010F4C00720F0C0072088C007205F
:10145000A4C5072034C00720E4C40720A0D107207A
:101460003CC80720ECC0072020BCBE002CC00720D1
:101470008CC1072098D1072030C00720B8C10720B1
:10148000C0C10720C4C10720E0C0072024C0072036
:1014900094C10720240000109F48006849F6991164
:1014A00088421CD19D48006820B901209B490860F2
:1014B000FFF7B2F905209A490860FFF702FD994845
:1014C0000068012806D0012096490860002096494E
:1014D000086003E09548006801F043F84CE7B4F574
:1014E000004F01D1FFF7DAFE8D48006802280ED1C7
:1014F00089480068B0F5704F02D1FFF72DFF3BE738
:101500008B48006840F400708949086034E78448DB
:101510000068052870D180480068B0F55A4F08D19E
:10152000FFF7E7FCFFF7CDFC8048006801F019F8F1
:1015300022E7794800684DF60121884205D1002054
:101540007C490860FFF7F3FB16E7B4F5614F02D161
:10155000FFF7D7FC10E7B4F5634F02D1FFF7D2FCD9
:101560000AE7B4F5654F02D1FFF7E7FC04E7B4F5ED
:10157000674F02D1FFF793FDFEE6B4F5644F02D149
:10158000FFF79AFDF8E6B4F5664F02D1FFF7AEFD1E
:10159000F2E6B4F5206F02D1FFF775FCECE6B4F586
:1015A0005D4F02D1FFF7B9FDE6E6B4F5684F02D111
:1015B000FFF787FEE0E6B4F5694F02D1FFF770FE52
:1015C000DAE6554800684DF60221884202D1FFF75D
:1015D0008DFED1E6504800684DF60321884202D1C5
:1015E000FFF793FEC8E64C4800684DF60421884298
:1015F00003D1FFF791FEBFE624E0474800684DF6AF
:101600000A21884202D1FFF79BFEB5E642480068F6
:101610004DF64021884202D1FFF788FEACE6B4F5D2
:10162000594F02D1FFF7A1FCA6E6B4F5584F02D1FD
:10163000FFF7BCFCA0E63E48006840F480603C49EF
:10164000086099E600BF97E610B53B48006800B90E
:1016500010BD3748006868BB384840783849096889
:10166000884204D0354840781F2800D027E033480E
:101670000078CC2817D100202B490860FFF76DFEB9
:101680002B48008800F40070B0F5007F06D0284891
:10169000008800F40060B0F5006F0FD124480068A6
:1016A000284908600AE02248006840F48070254913
:1016B000086003E01E4800682249086000BF1D481A
:1016C000006870B1204804680068204908601E481E
:1016D0000068402800D94024224618491C4805F0DB
:1016E000ABF800201349086000BF002116480068CD
:1016F000401E154A1060114A115413480068002812
:10170000F3D11148006813490860002008490860B7
:101710000949086000BF9BE728C0072088C107204F
:1017200024C0072094C10720F4C00720ECC0072084
:10173000FCC00720E0C00720DCC00720E4C407206D
:101740003CC80720F8C00720D4C00720E4C0072009
:10175000A4C40720D8C00720FC48406EFC49886319
:10176000FA48406E46F62B014843C00BF9494862DF
:1017700070474FF48070F749486070474FF48070AD
:10178000F4498860704710B5034609B9184610BD82
:10179000002923DD914200DD114643B10020EE4CCB
:1017A0002060EE480068401CEC4C206007E0002000
:1017B000EA4C2060E8480068401CE74C2060E7489D
:1017C0000068884202D10120E54C2060E2480068B0
:1017D000884227D10020E24C206023E04942914218
:1017E00000DD114643B1501CDB4C2060DB48006833
:1017F000401EDA4C206007E0501CD84C2060D648D0
:101800000068401ED44C2060D4480068884202D151
:101810000020D34C2060D0480068884202D10120CB
:10182000CF4C2060CE480068B1E70246CD488142E7
:1018300007D1CD480068CD4B18600020CA4B186016
:1018400004E0C94800681044C74B1860C7480068E6
:1018500070472DE9F84FC6490968880002F04AFA36
:10186000C449086008460068002803DB0120C2491B
:10187000086002E00020C0490860B648806E00F0B1
:10188000010000284CD0B348006F40F00100B1497E
:1018900008670846806B496B884226D9B7480068BC
:1018A00060B1AA48406EB64909684843C00AB549C4
:1018B0008861012008650020B0490860A348406E97
:1018C00046F62B014843C00BA24948639F48406E2F
:1018D0009E49096E401A46F62B014843C00B9D49AC
:1018E00088630020A84908601AE09848406E46F6D0
:1018F0002B014843C00B974988639448406E934935
:10190000096E401A46F62B014843C00B91494863C3
:1019100001209D4908609D480068401C9B49086063
:101920008B48016B9A48026897480068FFF72BFFC5
:1019300098490860084600688F49096848400121B5
:10194000C1EB400094490860944800680968084465
:1019500092490860924801688F480068FFF765FF68
:101960007A49886689480068282879DD00208749F7
:1019700008608C48007800F04000402870D174481E
:10198000806B850385480088404206B27048808E8F
:1019900007B2A846B146BA46424609FB0AF31846C2
:1019A000194600EB010BCDF800B000290DDDDDF884
:1019B00000B0834509DA00BFDFF8ECB14FF0010E4B
:1019C000CBF800E06FF0004B11E000290DDADDF8F4
:1019D00000B0834509DD00BFDFF8CCB14FF0010E48
:1019E000CBF800E04FF0004B01E0DDF800B05C46C2
:1019F00000BF1019002C08DD904206DA00BF6A49CA
:101A000001230B606FF000410AE0002C07DA9042DE
:101A100005DD00BF644901230B60D90700E00146E2
:101A20008C4600BF60464FF40041421800290ADD91
:101A3000824208DA00BF5C4C4FF00108C4F8008015
:101A40006FF000440EE000290BDA824209DD00BF8E
:101A5000554C4FF00108C4F800804FF0004401E0FD
:101A60001DE014462346181400BF00BF800038490B
:101A700088630846806B096C884203D93448006C3F
:101A8000334988633248806B3149C96B884203D23D
:101A90002F48C06B2E4988630020404908604148A8
:101AA000007800F0400040280BD12948806B27497E
:101AB00048660846406E46F62B014843C00B254950
:101AC00048622248406E2249096C884205D81F4866
:101AD000406E1F49C96B884205D23448006840F403
:101AE000804032490860BDE8F88F2DE9F047304862
:101AF00000683049096888427DDB00202C49086075
:101B00001349886B04F07AFE1148B0F85C0006B205
:101B10000F48B0F8600007B2FEF744FB0FFA80F8F8
:101B200007FB08F000F580421046114643180029D3
:101B300042DD834240DA00BFDFF86CC04FF001099C
:101B4000CCF800906FF0004C45E00000A0D10720D9
:101B50003CC8072000800B40ACC00720A8C007206D
:101B6000B0C0072000E1F505B8C00720B4C00720C9
:101B70001CC2072074C0072094C007208CC0072017
:101B8000E80000100080014088C00720BCC007208A
:101B900078C00720A4C00720A0C0072090C007205D
:101BA0000800001084C10720540100108CC10720D8
:101BB000CCC00720D0C0072000290BDA834209DD02
:101BC00000BFDFF824C44FF00109CCF800904FF0BB
:101BD000004C00E09C4600BF4FEA2C4500BF30049B
:101BE0002904421800290ADD824208DA00BFFE4BB0
:101BF00001271F6000E082E06FF000430AE0002947
:101C000007DA824205DD00BFF74B01271F60FB07A3
:101C100000E013461814F5490860F548006810B153
:101C2000F448446E02E0F348406E4442F2480088B3
:101C300003B2F148008806B227B206FB07F000F5B0
:101C400080421046114600EB010C00290BDD844553
:101C500009DA00BFDFF890834FF00109C8F800905F
:101C60006FF000480EE000290BDA844509DD00BF63
:101C7000DFF874834FF00109C8F800904FF0004876
:101C800000E0E04600BF4FEA2840400005B21804DB
:101C900029044218002908DD824206DA00BFD24E2C
:101CA000012737606FF000460AE0002907DA824218
:101CB00005DD00BFCC4E01273760FE0700E0164669
:101CC0003014CC4988650846806D496D884203D937
:101CD000C848406DC7498865C648806DC549096DCB
:101CE000884203D2C348006DC2498865C048006875
:101CF00008B9012000E00020BD49086004E0BF48A9
:101D00000068401CBD490860BDE8F0872DE9F84F28
:101D1000BB480068002807DDBA480068B849096870
:101D20000844B849086006E0B6480068B449096844
:101D3000401AB4490860B4480068B449884278D170
:101D4000B348007800F02000202873D1A948B0F8EB
:101D500044000004AF490860A648806C0968084345
:101D6000AC490860A748036808460268184611464F
:101D7000441A002907DD844205DD00BF9A4D012683
:101D80002E60F5070BE0002908DA844206DA00BF6E
:101D9000954D01262E606FF0004500E0254600BFFE
:101DA000E8109C49086008460068B0F5004F02DB67
:101DB00047F6FF7008609748006810F5004F02DA98
:101DC0009548944908608C480068850391480088CC
:101DD00006B28848B0F84C0007B2A846B146BA46E9
:101DE000424609FB0AF31846194600EB010BCDF8F1
:101DF00000B000290DDDDDF800B0834509DA00BF31
:101E0000DFF8E4B14FF0010ECBF800E06FF0004BCB
:101E100013E000290FDADDF800B083450BDD00BFC9
:101E2000DFF8C4B14FF0010ECBF800E04FF0004BEB
:101E300003E07CE05DE0DDF800B05C4600BF101917
:101E4000002C08DD904206DA00BF674901230B60D1
:101E50006FF000410AE0002C07DA904205DD00BF78
:101E6000614901230B60D90700E001468C4600BFA1
:101E700060464FF40041421800290ADD824208DA28
:101E800000BF594C4FF00108C4F800806FF00044C7
:101E90000DE000290ADA824208DD00BF524C4FF003
:101EA0000108C4F800804FF0004400E014462346C7
:101EB000181400BF00BF504908604E48406D0968C3
:101EC000B1EBA00F04DD4B48406D80104A4908601B
:101ED0004848006D48490968B1EBA00F04DA45484D
:101EE000006D801044490860434800688000424902
:101EF00008604448006840114849C86500204149CD
:101F000008604648C06D43490968C91101EB4101A9
:101F1000884206D24248006840F4004040490860C8
:101F200005E03F48006820F400403D490860FFF7A5
:101F3000DCFD3748007800F02000202803D12D4830
:101F4000806D36490866BDE8F88F3648006840F471
:101F500000303449C439C1F8C4000846D0F8AC0197
:101F600040F04040C1F8AC012F48406840F080404C
:101F70002D494860002088611E48806B46F62B0181
:101F80004843C00B284948621A48806B46F62B012B
:101F90004843C00B244908631648806D46F62B0160
:101FA0004843C00B204988631248806B1149896DF2
:101FB000401A46F62B014843C00B1B4948630846AC
:101FC000C06B6FF30900C86301204865084640688C
:101FD00016490843144948600648806D0649086060
:101FE0000448806D0D4923E054010010D0C0072043
:101FF000C8C007203CC807207CC00720CCC00720F1
:102000001CC20720C0C007200800001000E1F50531
:1020100084C10720C4C007200080FFFFA0D1072093
:102020008CC10720C4C00F4000800B40010101009B
:1020300008661A48806B486670472DE9F84301F03E
:102040007BFD47F2623015498863FFF77EFFFFF79B
:1020500090FB1348006805F067FE804605F082FD9E
:10206000064632460B4600200E4905F0D5F90446D7
:1020700001200D4A0D4B0090204601F0F3FE084868
:10208000006840080A4908600449896B094A1268D7
:102090005143C80AFEF782FCBDE8F8833CC807201C
:1020A000E40000100000F03F7B14AE47E17A843F6B
:1020B00078C00720E800001030B50022012103E0BD
:1020C000FE48405C0244491CFD480068801E88426E
:1020D000F6D8FB480068401EF84C245CF8480068BD
:1020E000801EF64D285C44EA0023981A30BD7047E4
:1020F00000B50AE0F3480068C1B2F1480268006820
:10210000401CEF4B1860ED488154EE48406900F0E8
:1021100001000028EED1EC48006846F2A811884280
:102120001ADD00BF0021E6480068401EE44A106046
:10213000E24A1154E24800680028F3D1E048006800
:10214000E2490860DF48806840F00200DD498860AD
:102150000020DD49086000BDDC480068D8490968F6
:10216000884208D1D848006820B1D7480068401C90
:10217000D5490860EFE7D2480068D4490860D048E4
:102180000068062804D3CE48007800F0010028B18A
:10219000CD480068401CCC490860DCE7CA480068AC
:1021A000D8B9C7480068012817D9C4480078CC2896
:1021B00007D1C248407802280FDDC04840781F2868
:1021C0000BD0C348006840F00500C1490860BE4814
:1021D0000068401CBC490860BDE7B9480068062893
:1021E00019D1B64880780A280FD0B4488078E02802
:1021F0000BD0B2488078E42807D0B0488078E62831
:1022000003D0AE488078E82817D1AF480068401C5A
:10221000AD4908609FE7AA48006808280DD1A74883
:102220008078E02803D0A5488078E42805D1A64826
:102230000068401CA44908608DE7FFF73DFF00B12E
:1022400089E70120A349086000209F49086000BF7A
:1022500081E770B59B4C646904F0400454B19E4C16
:10226000246804F400342CB99C4CE46D44F0080458
:102270009A4DEC659A4C246804B970BD914C646920
:1022800004F0400404B9F8E7934C246804F40034E3
:1022900004B1F2E70024924D2C600224914D2C6091
:1022A000DD24914D2C70914C24786C702C46617813
:1022B000002026E08E4C54F8203000221BE002F073
:1022C00001043CB91C88C4F30724874D854E366849
:1022D000AC5505E01C78844D824E3668AC551B1D0C
:1022E000814C804D2D68645D21447E4C2468641CC3
:1022F0007C4D2C60521C7F4C54F820409442DED818
:10230000401C7D4C2468A042D4D3C1F30724764DF1
:10231000744E3668AC55734C2468641C2955714C56
:102320002468A41C6F4D2C606F4C6B4D103D2C60CD
:10233000724CD4F82C416FF30B04704DC5F82C414E
:102340002C46D4F84C416FF30B04634D1C352C60C4
:1023500000246A4DC5F82841624C2468102C0BD922
:102360005D4C241F246844F01004C5F82C41644CD3
:10237000594D083D2C6008E0574C241F2468594DE6
:102380002D682C435D4DC5F82C41534C1C342468FA
:1023900044F00104594DC5F84C410024AD002C63B4
:1023A000584C2468042C10DA01244FF040256C604E
:1023B0004A4CA46D44F00804484DAC65464C246872
:1023C00044F001044D4DC5F83041434C203424689D
:1023D00044F00104494DC5F8504100BF4DE74A485B
:1023E000006840F000504849C439C1F8C4000320D7
:1023F0004649086001204149086300BF3F48006B1F
:1024000000F001000028F9D01A2001218140404A43
:10241000430942F8231000BF704710B54FF416412E
:10242000394B1B6843F00803374CC43CC4F8C43034
:10243000384B1B6843F05003364C2360364B1B6807
:102440009A088323354CE3601309B3FBF1F0030AC8
:102450006360C3B223602346DB6823F08003E3603C
:10246000C723A3600023636023469B6843F00803EF
:10247000A360284B5B6823F44043264C6360174BF2
:102480001B6843F40003154C23602346DB6943F4C7
:102490000003E36110BD10B54FF416421A4B1B68E0
:1024A00043F01003184CC43CC4F8C430194B1B69EA
:1024B00048F60A042343174C236131E0E4C40720A3
:1024C000D4C00720000001400CC10720D8C007205D
:1024D00010C10720DCC007203041005000C0092097
:1024E000F4C00720E8C0072024C507203CC8072007
:1024F00064C50720A4C50720F0C007200040005095
:10250000E4C5072094C10720C4C00F40C4C10F40D8
:1025100080E100E000C0024000C0072000C0004091
:10252000714B1B6899088323704CE3600B09B3FB64
:10253000F2F0030A6360C3B223602346DB6823F032
:102540008003E360C723A3602023E3640023636068
:1025500023469B6843F00803A36010BD63490860ED
:10256000704710B50246604B1B6899085F4BDB68EB
:1025700043F080035D4CE36032B1102A0ED0202A74
:1025800016D0302A23D119E00B094FF41644B3FBBF
:10259000F4F040F6A843564C236018E00B094FF4C2
:1025A000E134B3FBF4F040F24243514C23600EE0BF
:1025B0000B094FF4E124B3FBF4F008E00B094FF4EE
:1025C0006124B3FBF4F08C23494C236000BF00BFAF
:1025D000030A464C6360C3B223602346DB6823F0E2
:1025E0008003E36010BD4348006820F001004249C9
:1025F000C1F8300102208860086140483D49103927
:1026000008603A48091D086080023B49C1F82C0166
:102610000846D0F8300140F42860C1F8300108467F
:10262000D0F8300140F001003549086033482030CF
:10263000344908602D484860002088603248C860EE
:102640002E48103031490860284848602D4888607D
:102650002D48001DC8602848D0F8500120F0010026
:1026600024492031086004202349886008612848F3
:102670002049103108601D483030091D0860254888
:102680001D49C1F84C011B482030006840F652211A
:10269000084318492031086000201749C1F8480153
:1026A0000846D0F8900120F001001249603108601E
:1026B000102011498860086111480E4950310860A6
:1026C0000C48091D086013480B49C1F88C010846E5
:1026D000D0F8900140F42160064960310860002084
:1026E0000549C1F88801704700C00720000001407B
:1026F00000C10720304100500040005024C5072091
:1027000008C10720F4C507200C000004E4C5072019
:1027100004C10720009000800020E44908604FF0C9
:102720008040E34908624FF04050E0490864704738
:10273000E048006838B94FF08040DD4988630120E7
:10274000DC49086006E00020DA4908604FF080406C
:10275000D749C8637047D848D8490860D848086046
:102760001520D84948652020C864002088644FF4AB
:102770007A70D549086041F28830D4490860002059
:10278000D3490860D3490860D3490860D349086039
:1027900047F6FF70D24948618861FDF7D4FDFFF725
:1027A000BBFFC248006820F44070C049086008467A
:1027B000006C40F440700864BD48006840F01000B0
:1027C000BB490860102088610020B849C8600846ED
:1027D000C06C40F44020C864B548006A40F0007006
:1027E000B34908620846C06B40F00070C86300201F
:1027F000AE49C8600846C06C40F04070C864AC4840
:10280000006A40F08050AA4908620846C06B40F058
:102810008050C8630020A54988600846C06C40F01D
:102820004070C864A248006C40F48050A04908641D
:102830000846C06D40F48050C865FFF7D0FD02F037
:1028400006F9FDF7E7FCFFF7E8FDFFF724FE01F0CE
:10285000C3FD01F02CFE01F0DCFFFEF742F9FEF7AC
:10286000F8F8032002F00DF9FFF7BDFE01F08EFD30
:102870003C21084601F026FE00209A4908609A484B
:10288000C0689A49C86000F07DF9FFF7D6FB0120C7
:1028900097490860FDF7F8FD41F6846002F092FB6D
:1028A00002F09CFB02F0D6FB02F0DEFB4FF6FF705D
:1028B0008C49086020207E49C86100208D4908604D
:1028C0008D4908608D4908608D4908608D49086010
:1028D0008D4908608D4908608D4908608D49086000
:1028E00035E04FF6FF708C498A4A126841F82200A1
:1028F00001468A48874A126840F8221008468849EB
:10290000844A126841F8220000208649814A1268F0
:1029100041F82200002184487E4A126840F82210C3
:10292000002082497B4A126841F822000021804839
:10293000784A126840F8221000207E49754A1268D1
:1029400041F8220073480068401C724908607148D1
:102950000068FF28C5DD78A002F031F90020794930
:10296000086079A003F0D4FC00BF7648006820B16D
:1029700074480068401E7349086003F0ADFA02F025
:1029800046FF77480068642839D976480068401CBB
:10299000744908607448006801280BD10846006833
:1029A000B0F5FA7F06DD08460068A0F5FA70086009
:1029B00002F0FDFC6A4800686438694908604248D2
:1029C000006840B140480068401E3F490860102040
:1029D0003749886102E010203549C8613B480068EA
:1029E00048B13A480068401E384908604FF48050AA
:1029F0002F49C86503E04FF480502D49886502F0E7
:102A0000C3FA02F0F2F85948006800F0010000280B
:102A10004BD02F480068401C2D490860544800687E
:102A2000401C5349086053480068401C51490860E5
:102A300051480068401C504908600846006842F24E
:102A40001071884202DD00204B4908601848806DF3
:102A500040F00400164988654848C0684849086045
:102A6000FDF78AFE01F07FFDFDF765FF00F013FD25
:102A700000F0AAFB00F068F9FFF748F900F06CFBE2
:102A80001A49486001F021F801F086FBFFF730FB9E
:102A9000FEF7DAFDFFF7DDFB01203449086004484A
:102AA000C06D40F004000249C8655EE700C0024006
:102AB00000C0092050C107208F054B3F74C107207B
:102AC000CDCC4C3F34C4072030C1072034C107208F
:102AD00038C107203CC2072040C2072044C207205B
:102AE000BC19001084C107203CC80720A0D10720D2
:102AF00088C1072050C2072054C2072058C20720AF
:102B00009CC20720A0C20720A4C20720A8C2072099
:102B1000ACC2072028C1072058050010580D00102E
:102B200058010010DC190010DC1D0010DC21001021
:102B3000DC250010DC2900100A0D202E2E2E2E2E52
:102B40002E2E200024C407200A0D202E2E2E577270
:102B5000697465436F6E312E2E2E2E20000000000A
:102B600088C2072064C107202401001000800140B2
:102B700060C1072068C1072014C1072000C00B40B6
:102B800014C207202DE9F04F89B0FB48D0F8DC00D3
:102B9000FA49884203DA481CF749C1F8DC00F648D4
:102BA000806AF549C96A08444010F549086008463A
:102BB00000688001F3490860EF48D0F89C00642861
:102BC00004DCED48D0F89C000A2803DA2820EA4902
:102BD000C1F89C004FF0000A40E0E749D1F89C00A2
:102BE00005F08AF8064604F0BDFFCDE9060150461F
:102BF00005F082F8019004F0B5FF00224FF0804309
:102C0000CDE9020104F0BAFD0646DF4ADF4B04F0CD
:102C1000B5FDCDE90401DDE9062304F0FDFB8046A6
:102C200004F0C8FA044604F015FB8346D849584618
:102C300005F08EF8044605F023F8D64941F82A003D
:102C4000084650F82A00002806DA084650F82A00FC
:102C500000F5803041F82A000AF1010AC648D0F890
:102C60009C005045B9DCC449D1F89C0005F044F8FB
:102C7000804604F077FF064632460B460020C649E0
:102C800004F0CAFB04460020C44AC54B009020460D
:102C900001F0E8F8B848006A4000B7490862084601
:102CA000D0F89C004010BF49086009B0BDE8F08F23
:102CB0000146B148C06908B908467047AE48C069C6
:102CC000B84A1268904203DDB6480068AA4AD0614B
:102CD00041B10020B44A1060B4480068401CB34AB7
:102CE000106007E00020B14A1060AF480068401C47
:102CF000AD4A1060A048C069AC4A1268904202D147
:102D00000020AB4A10609C48C069A74A12689042F4
:102D100002D10120A64A1060A5480068CDE702460E
:102D2000A448814208D1A44800688014A34B1860CD
:102D30000020A14B186004E09F48006810449E4B9F
:102D400018609E48006870472DE9F05F8C48406825
:102D5000B0F5004F01DB002400E001249849C86869
:102D600001F012F89749086008460068002803DD62
:102D700001209549086003E04FF0FF309249086058
:102D80002046FFF795FF05464DB18E48006840424A
:102D90008C4908608C48006840428B4908608B4829
:102DA000006800287BD17448806A76490968B1EBD5
:102DB000801F49DD86480068002845D001208349EE
:102DC00008606D48B0F8800103B26B48B0F87C0130
:102DD00080490988081A06B203FB06F2104611461C
:102DE000471800290BDD874209DA00BFDFF8E8C188
:102DF0004FF00108CCF800806FF0004C0EE0002985
:102E00000BDA874209DD00BFDFF8CCC14FF00108C3
:102E1000CCF800804FF0004C00E0BC4600BF00BF83
:102E20005548D0F8DC0060446C49086001206C49CA
:102E300008706A48006880016A4908604E48D0F806
:102E400090014D49886057E14B48C06A4D49096877
:102E5000B1EB801F4ADA5E48006878BB01205B490D
:102E600008604548B0F8840103B24348B0F87C01DB
:102E700058490988081A06B203FB06F210461146A3
:102E8000471800290CDD87420ADA00BFDFF848C185
:102E90004FF00108CCF800806FF0004C10E0AAE081
:102EA00000290CDA87420ADD00BFDFF82CC14FF0A1
:102EB0000108CCF800804FF0004C01E016E0BC4661
:102EC00000BF00BF2C48D0F86C0160444649086040
:102ED0000220434908704448006880014149086065
:102EE0002548D0F890012449886005E12548076805
:102EF000354800880FFA80FC1F48008C0FFA80F8D4
:102F00003B460CFB08F21046114600EB0109002974
:102F10000BDD814509DA00BFDFF8BCA04FF0010BE3
:102F2000CAF800B06FF0004A0EE000290BDA8145C4
:102F300009DD00BFDFF8A0A04FF0010BCAF800B018
:102F40004FF0004A00E0CA46564600BF9819002ECE
:102F500008DD984206DA00BF1F4901220A606FF0BF
:102F6000004144E0002E41DA98423FDD00BF1A499B
:102F700001220A60D1073AE03CC8072034F3FFFF82
:102F8000A0D107204C000010F1D4C853FB21094008
:102F900000FEFF4604C607200000F03FFCA9F1D266
:102FA0004D62503F5C00001068000010640000108B
:102FB0006C00001000E1F50588000010840000108E
:102FC00090D1072050000010600000107000001029
:102FD00090000010980000105401001054000010E0
:102FE0007C0000107800001058000010014600BF5F
:102FF0006648016080E06648007800286DD064482B
:103000000078012834D1614803686248D0F88821EB
:1030100018461146461A00290ADD864208DD00BF1F
:103020005D4F4FF0010CC7F800C04FF000470DE0B6
:1030300000290ADA864208DA00BF574F4FF0010C28
:10304000C7F800C06FF0004700E0374600BF4F48A8
:10305000076000685149096888424DDA00205049EC
:1030600008604B4908704D4800684849086043E0D3
:10307000464803684748D0F8882118461146461844
:1030800000290ADD864208DA00BF434F4FF0010CE9
:10309000C7F800C06FF000470DE000290ADA864249
:1030A00008DD00BF3C4F4FF0010CC7F800C04FF0E7
:1030B000004700E0374600BF3448076000683749E2
:1030C0000968884218DD00203549086030490870D9
:1030D000324800682D4908600EE02E48406A3049A9
:1030E0000968884205DD2E480068401C2C490860AC
:1030F00002E000202B490860244800682A498842E1
:1031000002DD0846214908602048006827498842B6
:1031100002DA08461D4908602548007800F00800DA
:10312000082805D11948006880112249086004E088
:10313000204800688001154908601F4801681F4841
:103140000068FFF7ECFD1B498860BDE8F09F1B4855
:10315000006840428000704710B519480068401C64
:103160001749086008460068282801DB002008602D
:103170001449134A126851F8220001F006F9114867
:103180000F49096850F8210010BD00004C000010E4
:103190007C0000103CC8072054010010780000108B
:1031A0007400001070000010C0FF1F0000CDFCFF75
:1031B00084C10720A0D10720080000105000001093
:1031C0008000001004C607202DE9F0475A490989FC
:1031D000080400F09EFF5849886058484368084634
:1031E000826818461146441A002907DD844205DD2D
:1031F00000BF534D01262E60F5070BE0002908DAC9
:10320000844206DA00BF4E4D01262E606FF0004565
:1032100000E0254600BF4B4805614B48007800F0B0
:103220000200022865D1494805684648008A06B26E
:103230004248008907B22B4606FB07F210461146AA
:1032400000EB010C00290BDD844509DA00BFDFF833
:10325000F0804FF00109C8F800906FF000480EE0D0
:1032600000290BDA844509DD00BFDFF8D4804FF078
:103270000109C8F800904FF0004800E0E0464446DD
:1032800000BF1819002C08DD984206DA00BF2C494F
:1032900001220A606FF000410AE0002C07DA984230
:1032A00005DD00BF264901220A60D10700E0014682
:1032B00000BF264801602148008A24490968B1EB13
:1032C000004F04DD1D48008A0004204908601B48A7
:1032D00080891E490968B1EB004F04DA17488089DC
:1032E00000041A4908601948006800141549C860AC
:1032F00004E0144880890004144908601148C0683B
:1033000046F22221884205DA0E48C06842F22221A4
:1033100088420FDC0B48C0680D49884204DA09482E
:10332000C0680C49884205DC0B48006840F4005036
:1033300009490860BDE8F08790D107203CC8072004
:1033400054010010A0D1072084C107207CC10720B0
:1033500023C2FFFF2382FFFF8CC107202DE9F04726
:1033600005462E46FE48D0F83001B04202DAFC484D
:10337000D0F83061002400E0641CF948FC3050F8BB
:103380002400B042F8DBF649FC3151F82410881BC8
:1033900004F0B2FC8146F34951F8240004F0ACFC7F
:1033A0008246494604F0D4FC8046EF4850F8241089
:1033B000404604F099FD0746384604F061FCBDE83C
:1033C000F0872DE9F047E9480568E948006878B3D7
:1033D000E348D0F8C801A84202DAE148D0F8C85161
:1033E000002400E0641CE048603050F82400A8424B
:1033F000F8DBDD49603151F82410481B04F07CFCF7
:103400008046DC4951F8240004F076FC81464146B0
:1034100004F09EFC0746D448983050F824103846F3
:1034200004F062FD064604F02BFCD34908602EE050
:10343000FFE7CB48D0F83C02A84202DAC848D0F8EF
:103440003C52002400E0641CC748D43050F82400EB
:10345000A842F8DBC449D43151F82410481B04F0C9
:103460004BFC8046C54951F8240004F045FC8146D8
:10347000414604F06DFC0746C14850F82410384618
:1034800004F032FD064604F0FBFBBB490860BA4875
:103490000068BDE8F0872DE9F041002407E0B94855
:1034A00050F82420B848211D40F82120641C022C2B
:1034B000F5D3B6480068B649884204D1B5480068DB
:1034C000401CB4490860B348006804282DDD002082
:1034D000B0490860B0480068401CAF490860A34884
:1034E0000068AE490860AE48006849F6404190FB6C
:1034F000F1F09E49086008460068A84909688842BA
:1035000004DDA8480068401CA64908609748006888
:10351000A2490968884204DAA2480068401EA1490D
:10352000086000209E49086008E097488038D0F87D
:1035300090009B49096808449949086096480068CA
:103540000A2813D100209449086096480068002892
:1035500002DD01208649086092480068002802DAEE
:1035600000208349086000208E4908608E4800686A
:10357000002879D08848006803287FDD00208A4928
:103580000860774890F8F80078B1754890F8F8002E
:1035900004280AD0724890F8F800062805D073482D
:1035A0000068FFF7DBFE81490860FFF70AFF6C48FF
:1035B000B0F8800103B26A48B0F87C016B49098811
:1035C000081A05B203FB05F21046114646180029F9
:1035D0000ADD864208DA00BF754F4FF0010CC7F8CC
:1035E00000C06FF000470DE000290ADA864208DDCE
:1035F00000BF6F4F4FF0010CC7F800C04FF00047FD
:1036000000E0374600BF00BF5548D0F8DC00384422
:10361000684908605248B0F8840105B25048B0F8D3
:103620007C0152490988081A03B205FB03F21046CF
:103630001146461800290ADD864208DA00BF5C4FB1
:103640004FF0010CC7F800C06FF000470EE00029F2
:103650000BDA864209DD00BF554F4FF0010CC7F869
:1036600000C04FF0004701E008E0374600BF00BF50
:103670003B48D0F86C0138444F4908603B49096821
:103680004E4A1268881A002801DB014600E04142D8
:10369000334AD2F80422914205DD34480068474994
:1036A0000860FFF78EFE38488038D0F89000444913
:1036B000884216DB34488038D0F8900043F2C821A5
:1036C00088420EDC30488038D0F894003C4988426B
:1036D00007DB2D488038D0F8940043F2C821884297
:1036E00005DD3848006840F48050364908602649B6
:1036F0008039D1F89020D1F89410501A002801DBBD
:10370000014600E0414240F21452914205DD2D484D
:10371000006840F400602B490860BDE8F0812DE9A5
:10372000FC410F48D0F87801801003B20C48B0F883
:103730007C010E490988081A05B203FB05F000F563
:103740008042104611464618002940DD86423EDA86
:1037500000BF174F4FF0010CC7F800C034E0000065
:103760003CC8072004C8072070C907209800001033
:103770009000001094C7072094000010CCC70720C9
:103780007CCA072090D1072020D207200800001013
:1037900000E1F505A8000010AC000010B800001012
:1037A000A40000109C000010B4000010A000001045
:1037B000540100105400001058000010B000001018
:1037C0003CF6FFFF8CC107206FF000470DE0002999
:1037D0000ADA864208DD00BF134F4FF0010CC7F82C
:1037E00000C04FF0004700E0374600BF3C1400BF68
:1037F0000E480068204401900D4800682044009065
:1038000043F6FE7101A803F04DF943F6FF716846D7
:1038100003F048F9019880000649C86300988000C9
:103820000864BDE8FC8100005401001080C007203E
:1038300084C007203CC80720AA48006800B9704728
:103840000020A9490860A9490860A6490860A8495C
:103850000860A849086000BFF1E710B5A4480078E7
:10386000C0F3C01020B90020A1490860FFF7E4FFB1
:10387000A1480068A149096888420CD0FCF7F8FF0C
:1038800048B19E4800689C490860084600680128C5
:1038900001D19B49086010BD9A48006888B19A48D8
:1038A0000068401E984908600846006800B17047EB
:1038B00000209449086095480068401C93490860BE
:1038C00009E093489149096850F821008E49086041
:1038D00001208C49086000BFE9E78A480068A0B170
:1038E00089480068401E884908600846006800B1A1
:1038F000704700208349086084480068401C834961
:1039000008601020834988610CE081487F4909687C
:1039100050F821007C49086001207A490860102095
:103920007C49C86100BFE3E770B5764800680028AD
:1039300070D079480068002820DD78480368764810
:103940000268184611464418002908DD844206DA48
:1039500000BF734D01262E606FF000450AE000297C
:1039600007DA844205DD00BF6D4D01262E60F507A4
:1039700000E0254600BF694805601FE0674803680E
:103980006548026818461146441A002907DD84423A
:1039900005DD00BF624D01262E60F5070BE0002912
:1039A00008DA844206DA00BF5D4D01262E606FF012
:1039B000004500E0254600BF5848056052480068B1
:1039C000401E514908600846006800B170BD0020E3
:1039D0004C4908604D480068401C4C4908604F48FD
:1039E000006842F21071884206DB4248006840F0ED
:1039F000010040490860E9E74A480068401E49491B
:103A000008600846006800B9E0E700203F49086008
:103A10000DE0FFE73E483D49096850F821003A496A
:103A2000086001203749086000203C49086000BF59
:103A3000CCE710B52C48006800B910BD2B480068D1
:103A400050B901203749086000202E4908602F49ED
:103A5000086001202549086033492C4A126851F852
:103A6000220080472748006800B1E6E72748006841
:103A7000032804D300201C4908601C49086000BFCB
:103A8000DBE710B52948006800B910BD2848006878
:103A900038B900201B4908601C49086001202449EE
:103AA00008602449194A126851F8220080471548D5
:103AB000006800B1E9E71548006820B100201B4903
:103AC00008601B49086000BFDFE710B5FFF7B1FFD2
:103AD000FFF7C3FEFFF7B0FEFFF7D3FFFDF767F96F
:103AE00010BD0000C0C10720B8C10720BCC107201D
:103AF00084C10720B4C10720E4C1072094C1072076
:103B0000F4C00720D0C10720D4C10720CCC10720B2
:103B1000A8C1072000C009201CC20720E8C1072057
:103B200054010010D8C1072098C10720C4C1072044
:103B3000C8C10720A4C107202DE9D043FE49896BE5
:103B40004FF44072B1FBF2F1FC4A11601146098852
:103B50000EB24FF4C07706FB07F319461A4601EB85
:103B6000020C002A0BDD8C4509DA00BFDFF8D08398
:103B70004FF00109C8F800906FF000480EE0002AED
:103B80000BDA8C4509DD00BFDFF8B4834FF0010983
:103B9000C8F800904FF0004800E0E046404600BF03
:103BA00000BFE549896B091AB1F5C07F04D9E34923
:103BB0000968491CE14A1160E04909686FF0004258
:103BC000B2FBF1F400200AE00021DE4A42F82010A6
:103BD000DD4A42F82010DD4941F82040401CD74919
:103BE00009688842F0D3D549096846F62B02B2FB32
:103BF000F1F1D74A116011460968491C1160BDE80E
:103C0000D0832DE9F041064600273C463D463A4622
:103C10003B46CC48CF4F3F6840F827607042CA4FC0
:103C2000DFF830C3DCF800C047F82C00002114E0B6
:103C3000C64850F82100C34F57F8217080FB077029
:103C4000BA184341C14850F82100BF4F57F82170BE
:103C500080FB07703C194541491CB8480068814207
:103C6000E6D3BD4F3B60BD480260501BBC4FDFF840
:103C7000E4C2DCF800C047F82C003846B54F3F6876
:103C800050F82700C0F10000B64FDFF8C8C2DCF8DA
:103C900000C047F82C004FF000021446254611469C
:103CA00013E0AA4850F82100AD4F57F8217080FB6F
:103CB00007078218A54850F82100AA4F57F821702D
:103CC00080FB07703C194541491C9C4800688142B3
:103CD000E7D3A0480068401C9E4F386097480068B2
:103CE000401E3F68B84202D200209A4F3860501BF5
:103CF000BDE8F081F0B505460026334634469A48C3
:103D00000068022802D90020974E30609748964EEE
:103D1000366840F826509448026800269448924F2E
:103D20003F6840F8276000211AE0924850F82100CF
:103D30008E4E56F822607043C31844EBE0748E48F0
:103D400050F821008A4E56F8226000FB06F0C31896
:103D500044EBE074A2F10100021E00DA0222491CC9
:103D60000329E2D3980B40EA8440814E7E4F3F689E
:103D700046F827007C4806680068401C7A4F386087
:103D80007B4850F82600F0BDF0B5054600263346C6
:103D900034467A480068022802D90020774E306005
:103DA0007748764E366840F82650744802680021FD
:103DB0001AE0744850F82100714E56F822607043A2
:103DC000C31844EBE074704850F821006F4E56F869
:103DD000226000FB06F0C31844EBE074A2F101007E
:103DE000021E00DA0222491C0329E2D3980B40EAA2
:103DF0008440664E614F3F6846F827000020034626
:103E0000044600211AE05F4850F821005F4E56F842
:103E100022607043C31844EBE0745B4850F8210003
:103E20005B4E56F8226000FB06F0C31844EBE074CA
:103E3000A2F10100021E00DA0222491C0329E2D38A
:103E4000980B40EA8440524E4C4F3F6846F827009A
:103E50004A4806680068401C484F38604C4850F893
:103E60002600F0BD2DE9FF5F88B000204949DDE95B
:103E70000A2303F083FC0022474BCDE9060103F03F
:103E80007BFD06460F4632463B463046394603F038
:103E900075FC04460D46414A414BDDE9080103F03B
:103EA0006DFCCDE9040103F037F900224FF08043A7
:103EB000CDE9060103F062FC82468B4652465B4622
:103EC00000204FF0804103F063FD52465B46CDE990
:103ED00006013046394603F051FC00222E4BCDE955
:103EE000000103F049FD22462B46CDE9020103F013
:103EF000E3F9CDE90401DDE9062303F08DFA8046FC
:103F00008946169810B101287DD19CE042464B4667
:103F10000020214903F03CFD0022224BCDE90401A1
:103F200003F02CFCCDE9060103F0CEFB1549086037
:103F300032463B46404637E03CC80720E4000010CC
:103F400054010010E8CA0720F4CB072018CF07203F
:103F5000E8000010EC000010C4000010C8000010C1
:103F600000CD07200CCE0720F000001054D0072011
:103F700060D007203CD0072048D00720F400001074
:103F80006CD0072024D0072030D0072078D007201D
:103F900084D00720000008400000F03FF1D4C8534F
:103FA000FB2119400000D040494603F0F1FC524685
:103FB0005B46CDE9020103F0E1FB00226D4BCDE948
:103FC000040103F0DBFBCDE9060103F07DFB6A4948
:103FD000486042464B462046294603F0D9FC002261
:103FE000644BCDE9040103F0C9FBCDE9060103F000
:103FF0006BFB6149886000206049086052465B465F
:104000003046394600E080E003F0B8FB0022594B0F
:10401000CDE9040103F0B2FBCDE9060103F054FB46
:104020005649486085F000400022524BCDE90440DB
:104030002046059903F0A2FBCDE9060103F044FBFD
:104040004E49886061E042464B4600204C4903F0EF
:104050009FFC0022474BCDE9040103F08FFBCDE923
:10406000060103F031FB4749086032463B464046B3
:10407000494603F08DFC52465B46CDE9020103F050
:104080007DFB00223B4BCDE9040103F077FBCDE93A
:10409000060103F019FB3B49486042464B46204667
:1040A000294603F075FC0022324BCDE9040103F0F0
:1040B00065FBCDE9060103F007FB3249886000206B
:1040C0003149086052465B463046394603F056FB9C
:1040D0000022284BCDE9040103F050FBCDE9060195
:1040E00003F0F2FA2849486085F000400022214B95
:1040F000CDE904402046059903F040FBCDE90601D7
:1041000003F0E2FA2049886000BF00BF0CB0BDE8B0
:10411000F09F10B501461D481D4A126850F8220054
:10412000C3171C4AD2E90042201A62EB0302194B62
:1041300005C31648164A126840F822101548D0E9FF
:1041400000305B1840EBE170124AC2E900301048C1
:10415000006800F101000E4A10601046007800F07F
:104160003F0010600B4A05CA4FEA905040EA822097
:1041700010BD00000000D04024D0072030D0072020
:104180000000F03F3CD0072048D0072090D0072007
:1041900000010010F8000010CF49096801B1704714
:1041A000CE490968491ECD4A116000290BDA4FF447
:1041B0007A7111600121C84A11601021C84A11604A
:1041C0002C219161EBE7C649096801F0080101B9AA
:1041D000E5E7C3494868202869D006DC082809D0EB
:1041E00010281CD018286CD127E0282833D030287C
:1041F00067D15DE00021BB4A11604FF47A71B74A84
:104200001160B8490A680968491CB64B1960B6497B
:1042100051F82210B24A91602821916151E0B149D0
:104220000A680968491CAF4B1960AF4951F8221060
:10423000AB4A91602821916143E0AA490A68096864
:10424000491CA84B1960A84951F82210A44A916052
:104250000821916135E0A349096806290AD10121A5
:104260009D4A116010219E4A11604FF496719F4A39
:10427000516718E09B490968032906D12021984A13
:104280001160C821994A51670DE096490A6809688A
:10429000491C944B1960944951F82210904A91603E
:1042A0006421924A516708218D4A916109E000BF5B
:1042B00010218B4A1160282191610121864A1160E9
:1042C00000BF00BF00BF6AE78948006820F0010016
:1042D000874908608748C06800F0100028B1084688
:1042E000006840F0010008601EE048F201008149CA
:1042F00088608148007800F0010050B1302088606B
:104300007A48C068404247F6FF710844794988609E
:104310000AE0312077498860744800684FF6F071F0
:1043200001EA400073498860704700BF704909681E
:1043300021F001016E4A11606E49C96801F0100157
:1043400079B11146096841F0010111606949C968F4
:1043500001F00101C1B91146096841F00101116084
:1043600012E064498968654A116062498968516050
:1043700060498968916001E05E4988685D49C96863
:1043800001F004010029F7D1704770475C480068CC
:1043900040F400205A49C439C1F8C4005948406863
:1043A00020F07070574948600846406840F0A0709F
:1043B00048606C204A4988618020486108615E201D
:1043C00049490860002048605C20C86000200861FE
:1043D000402043490860704700BF4949096841F4DB
:1043E0000011474AC43AC2F8C4101146D1F8AC11C2
:1043F00021F44061C2F8AC114149E8310968C2F8C2
:10440000AC114049096821F040413E4A1160114613
:10441000096841F0004111601146496821F03F01EF
:1044200051601146496841F0280151601146096CFC
:1044300021F0404111641146096C41F04041116482
:104440001146496C21F03C0151641146496C41F020
:104450003C01516440F20F31264A11600221116182
:10446000516000BF2349C96801F010010029F9D14A
:1044700001E0204988681F49C96801F0040100294A
:10448000F7D12149096841F480311F4A1160114672
:10449000896941F4803191611146096841F4000154
:1044A00011601146C96941F40001D1617047154896
:1044B000406840F4001013494860002013498860A8
:1044C00048607047084A906051612022044B1A608E
:1044D0000022014B1A607047040100101001001007
:1044E00000C001400C01001040D20720A0D10720DD
:1044F00008010010008008400000001090D1072043
:10450000C4C00F4000C0024000C0092000C00840E5
:1045100010B5036843FA01F202FA01F30468E31AE2
:10452000036010BD2DE9F0470446894684FB09501D
:104530000646DE480268D3172846314602F03AF9AB
:10454000054609F1010084FB00708046D7480268E7
:10455000D3173846414602F02DF90746D4490F607B
:104560002846BDE8F08710B5D2480068D2490968EE
:10457000401AD2490860CF480068CF490860CF4848
:104580000068B0F1804F06DBCC4800686FF0004156
:10459000401ACA490860C9480068B0F1404F06DCBB
:1045A000C64800686FF000410844C4490860C34928
:1045B00009888804FFF725FBC1490860C1480068E5
:1045C000002875D0012874D1BF480068002872D037
:1045D000BE480168BA480068FFF7A4FFBC490860FC
:1045E000B44800684FF6FF7101EA1041B948C0F8BD
:1045F0008810B048008881B2B648C0F88C10B64820
:104600000068B34909680844B3490860B348D0E971
:104610000031AF480068C21718185141AF4A03C2B1
:10462000AD480068AE490968401AAA4908670846BB
:10463000006F0014C8666FF00040A4490860A748E6
:10464000D0E90010A34A9832C2E900100020A44922
:104650000860A4480068062806D0A2480068072819
:104660000AD1A148006838B100209B4908600021A8
:104670009A4A1160516003E010219748FFF748FF04
:104680008F4800688A490968401A91490860924831
:10469000006809680844904908609048D0E90031F2
:1046A0008B480068C217181851418C4A03C213E0A6
:1046B00017E0A4E0FFE788480068814909680844DA
:1046C000854908608548D0E900317D480068C217F7
:1046D00018185141814A03C279480068834908602B
:1046E0008DE08348006800F00400002848D081482D
:1046F000006881490968401A804908607D4800685F
:104700007D4908607D480068B0F1804F06DB7B483A
:1047100000686FF00041401A7849086077480068E7
:10472000B0F1404F06DC754800686FF00041084466
:10473000724908607248406820B170480068714949
:10474000086004E06D48006840426F4908606848AE
:10475000006800F0080068B16B4800686B490860A9
:104760006948006867490968401A69490968084446
:10477000674908605E48006820F00C005C490860EA
:1047800051480068D0B36FF0004050490860494874
:1047900000684FF6FF7101EA10414E48C0F88810DA
:1047A0004448008881B24B48C0F88C1057480068D4
:1047B00058490968401A5849096808445649086028
:1047C00053480068434948670846406F52490968A2
:1047D00000EB61003F49486700204D490860012116
:1047E0004D48FFF795FE494800684A49086045482A
:1047F00000683849C86744480068886700BF00BF40
:104800002E480068334948652D48006800148865C3
:1048100010BD10B54148006840F480203F49C439BC
:10482000C1F8C4000846D0F8AC0140F00100C1F85E
:10483000AC013B48C06820F482403949C860084652
:10484000C06840F48240C8600846C06C35490843DF
:104850003349C86434482A4908610220C8630F20DC
:1048600008600020886041F6FF70304908602F49D9
:10487000103908601F200021002807DACA06140E2C
:104880002B4A00F00F031B1FD45403E0CA06130E7B
:10489000284A135400BF1F20012181404209920081
:1048A00002F1E022C2F8001100BF10BD1400001098
:1048B00010C2072014C20720F0C107201CC2072025
:1048C00020C2072088C107201C0000102000001013
:1048D00008C20720A0D10720FCC1072000C2072082
:1048E0008C00001094C10720240000100CC2072087
:1048F0002800001018C20720F4C10720F8C10720C3
:1049000000C00B4034C2072030C2072028C2072055
:104910002CC2072038C2072024C20720C4C00F4081
:1049200000C0024000C30300FEFFFF7FE8CF0B4042
:1049300018ED00E000E400E000216E4A116043F64B
:10494000E82151600121916011468968C2F89011F7
:10495000694911616949D1604FF4C8415161002131
:1049600091610521D161116247F6C041916242F621
:104970001961D1621E215162042111630902516340
:1049800000219164032151645D49D1646421116562
:1049900042F22671516544F2D801916343F6F04129
:1049A000D16344F2C04111644FF4A05191654FF4BA
:1049B000FA71D1654FF4C871116641F658315166EC
:1049C00000219167D167C2F88010C2F88410C2F844
:1049D0008810C2F88C10C2F89010C2F89410C2F877
:1049E0009810C2F89C10C2F8A010C2F8A410C2F827
:1049F000A810802191660021D1664FF48071116763
:104A00000021516700200AE04FF480423949C43147
:104A100041F820200022183941F82020401C0628A7
:104A2000F2DB47F6FF71334AC2F888114FF4E651C2
:104A3000C2F8DC1047F22021C2F86C113C21C2F808
:104A4000E010C2F8E4100121C2F8F01070472D48C0
:104A5000006820F001002C49C1F87001082088602E
:104A60000861C0032749103908602248091D086001
:104A700026482449091F086001202349C1F8700114
:104A8000704700B50346032B2BD100BF1D480068BB
:104A900000F400300028F9D11B48806900F00800BC
:104AA00030B11948006940F008001749086115E065
:104AB0001548406900F0080068B11348806840F06C
:104AC0000800114988600B48D0F8E80045F2AA5167
:104AD000884203D100BDFFF7BAFFFBE7FFF72CFFC9
:104AE00001E0FFF729FF034890F8F000084908604B
:104AF00000BFEFE73CC807201DBCFFFF6480FFFF3D
:104B000030F8FFFF7041005000400050AB00448C73
:104B100030C007205449096841F01001524A116021
:104B20001146096841F04001116083214F4AD1606C
:104B300027200146C21700EB126212124B4B5A603B
:104B4000C21700EB12621212A0EB02221A600321BC
:104B50001A46D16006219160704744490860704749
:104B6000002043490860434908607047404909688C
:104B7000491C3F4A116011460988C1F309011160BF
:104B80003D4A3B4B01681B6842F82310704730B523
:104B9000002211E0364B1B685B1C354C236023461A
:104BA0001B88C3F30903236010F8013B324C304DDE
:104BB0002D6844F82530521C8A42EBD330BD10E0FA
:104BC0002B490968491C2A4A116011460988C1F31A
:104BD0000901116010F8011B274A254B1B6842F898
:104BE000231001780029EBD1704722480068204942
:104BF0000968884214D01D48406900F0200078B14F
:104C00001C480068401C1B49086008460088C0F327
:104C1000090008601848096850F821001349086025
:104C2000704700201549086015490860704714480E
:104C3000006812490968884201D00C4840697047F1
:104C40000BE00A4800680F490C4A126841F822003C
:104C50000A480068401C094908600448406900F09F
:104C600001000028EDD1704700C0024000C00040A4
:104C7000140100101801001058D207201C01001068
:104C80002001001058E207200020A6490860A6482D
:104C9000C06880B2A549086008460068A449096850
:104CA000401AA0490860A1480068A14908609D48D1
:104CB000006810F5805F05DC9A48006800F58030D8
:104CC0009849086097480068B0F5805F05DB954813
:104CD0000068A0F5803093490860924800684FF65C
:104CE000FF7108449349944A126841F822008E48A3
:104CF000406820B18B4800689049086604E0894804
:104D0000006840428D49C8658D48006801287DD102
:104D100088488949096850F821008A490968084487
:104D200088490860844800780838C0B2814951F841
:104D3000200084490968081A82490860084600680A
:104D40004FF6FF71084480497B4A126841F82200FF
:104D500078487949096850F821007C490968084475
:104D60007A490860744800781038C0B2714951F827
:104D7000200076490968081A7449086008460068E6
:104D80004FF6FF71084472496B4A126841F82200DD
:104D900068486949096850F821006E490968084463
:104DA0006C490860644800782038C0B2614951F805
:104DB000200068490968081A6649086008460068C2
:104DC0004FF6FF7108445D494866624800684FF637
:104DD000FF7101446048584A126840F82210554853
:104DE0005549096850F821005C49096808445B4945
:104DF0000860514800781038C0B24E4951F8200080
:104E000056490968081A5549086000E05CE04A48BC
:104E100000782038C0B2474951F820004F4909684E
:104E200008444E490860444800783038C0B24149CF
:104E300051F8200049490968081A4849086008469D
:104E400000684FF6FF71084445493B4A126841F833
:104E5000220008463849096850F8210000F58030E2
:104E60003D49354A126851F82210411A3D48324AEC
:104E7000126840F8221038482F49096850F821007C
:104E800050B135482C49096850F821003649096865
:104E900008443549086043E02748007800F01F00C7
:104EA00038B9314800682549C86600202E49086095
:104EB00036E029482049096850F821002A49096844
:104EC000081A294908602BE01B480068FF2827D1F1
:104ED00001201B4908600020244908601CE04FF6AF
:104EE000FF701449214A126841F82200014618480F
:104EF0001E4A126840F82210084617491B4A1268D9
:104F000041F822001649194A126841F82200174850
:104F10000068401C1549086014480068FF28DEDD61
:104F20007047000048C2072000C00B406CC2072039
:104F300070C207205811001094C2072034C4072003
:104F40004CC2072050C20720580D001054C2072041
:104F50005805001058C20720580100105CC20720F5
:104F6000580900105815001064C2072068C20720B5
:104F70000F48006840F001000D49086070470C4878
:104F800000680B49086070470A48006864280ED919
:104F90000948006801280AD100200749086040F646
:104FA000B8300649086041F288300549086070470A
:104FB00074C2072038C10720C4C1072030C10720B0
:104FC00034C1072010B504463D48846103203C49A4
:104FD0004861022000F068F8002010BD0120384927
:104FE0004860704710B54FF480303649C861C00141
:104FF000886135480068401C3349086008460078DD
:1050000008600846007800F01F00304908602E480C
:10501000007800F03F002E4908604FF480302949A5
:105020008861C001C861FFF72FFEFBF7F0FA29483D
:105030002549096850F82100274909680844A0F566
:105040007F40FF382449086000F057F801201C49D0
:10505000086010BD10B5FA2020498861032048611E
:1050600000F022F8012010BD01201C494860486072
:10507000704710B501201949086019480068401CA4
:105080001749086017480068401C16490860164810
:105090000068401C1449086014480068401C13490B
:1050A0000860FBF709FA10BD00F01F0201219140D2
:1050B0004209920002F1E022C2F80011704700009C
:1050C0000080004000C0092094C2072090C2072041
:1050D00098C207205801001044C207200000094070
:1050E00078C207207CC2072084C2072088C207201C
:1050F0004FF4001076494860704776498968764ACF
:10510000116174498968D1607249896891607149F7
:10511000896851606F4989681160114609696F4A51
:10512000916045F255516B4A9160916091606C4974
:10513000097801F0010129B130219160664949697E
:10514000916005E03121634A91606349896991600A
:105150006449654A126851F82210C1EBC10101EBA4
:10516000810145F234321144604A116001E059492D
:1051700088685849C96801F004010029F7D15649E7
:1051800009685B4A5B4B1B6842F8231052494A6826
:105190005949584B1B6841F823204F498A685749A1
:1051A000544B1B6841F823204B49C968544A514B62
:1051B0001B6842F8231048490A6952494D4B1B6845
:1051C00041F823204B4A126851F822104E4A1268C7
:1051D00011444D4A1160474909782039C9B2494AFA
:1051E00052F82110484A1268511A474A1160114674
:1051F0000A6846493F4B1B6841F823203E493D4A17
:10520000126851F82210424A12681144404A116053
:10521000384909782039C9B2374A52F821103C4A36
:105220001268511A3A4A11603449324A126851F8E8
:105230002210384A12681144364A11602D49097803
:105240002039C9B22D4A52F82110324A1268511A37
:10525000304A11602A49274A126851F822102E4A12
:10526000126811442C4A1160224909782039C9B2C8
:10527000234A52F82110284A1268511A264A11600E
:105280001B491C4A126851F82210244A1268114422
:10529000224A1160174909782039C9B2144A52F8D4
:1052A00021101E4A1268511A1C4A116070474FF4AF
:1052B00080301B49C861C00188610846806D40F09C
:1052C000040088654FF480308861C001C861704770
:1052D00000C0024000800840BC19001090D1072097
:1052E00090C20720B0C2072098C2072000C0084023
:1052F000DC19001094C20720DC1D0010DC21001016
:10530000DC250010DC2900109CC20720DC2D0010D9
:10531000A0C20720A4C20720A8C20720ACC2072051
:1053200000C0092070B5024601240120002302E0DC
:10533000155D2B44641C8D1EA542F9D8555DC3F341
:105340000726B54208D00020FB4D95F8585005F0CF
:105350000205F94EB565B5654D1E555DDEB2B54227
:1053600000D00020C3F307268D1E56554D1E535501
:1053700070BD10B5F04890F84400F0490870EE4850
:1053800090F848004870EC4890F854008870EA485B
:1053900090F84C00C8700020087148710821E74857
:1053A000FFF7C0FF0821E54800F0E2FF10BD2DE93E
:1053B000F04F93B04FF08040E1498863DE48806849
:1053C000000BE049B1FBF0F0DB498866FF2048653F
:1053D0000846B0F86800C0F30727084690F86860F0
:1053E000B0F85C00C0F30729084690F85C80B0F87C
:1053F0006000C0F3072B084690F860A0B0F8640086
:10540000C0F307201190084690F8640012900846F7
:10541000B0F86C00C0F307200F90084690F86C00BD
:105420001090C9480088C0F30725C74804788088D1
:10543000C0F307200490C44800790890C24800894E
:10544000C0F307200390C048007A0790BE488089C7
:10545000C0F307200290BC48007B0690BA48008A3F
:10546000C0F307200190B848007C0590B648008B37
:10547000C0F307200990B448007E0A90FF200D90E9
:105480000E900B900C90084690F84400AB490870C1
:10549000A94890F848004870084680F8029080F8C3
:1054A000038080F804B080F805A0119888711298E4
:1054B000C8710F980872109848720D9888720E98EB
:1054C000C8720B9808730C98487308468773C673A4
:1054D000994890F854000874974890F8540048741C
:1054E000780888740846C674934890F85400087584
:1054F000914890F854004875099888750A98C875BD
:105500008D4890F8540008768B4890F854004876FF
:1055100008468576C476057744778577C47780F822
:10552000205080F8214080F8225080F8234000204D
:1055300081F8240081F825007F4890F8540081F814
:1055400026007D4890F8540081F827007A4890F8AA
:10555000540081F82800784890F8540081F8290018
:105560002C217648FFF7DEFE2C21744800F000FF66
:105570004FF080407249C86313B0BDE8F08F70B53A
:105580006D4890F844006D4908706B4890F84800E9
:105590004870694890F8400088706C48007800F0C6
:1055A000800008B1012400E000246848007800F081
:1055B0001000002850D100256448007800F00F004A
:1055C00008283CD2DFE800F0040A11181F262D3409
:1055D0005948006820435849086030E05648006840
:1055E00040EA44005449086029E05348006840EA12
:1055F00084005149086022E04F48006840EAC40036
:105600004D4908601BE04C48006840EA04104A49D4
:10561000086014E04848006840EA441046490860C1
:105620000DE04548006840EA84104349086006E000
:105630004148006840EAC4103F49086000BF00BF0D
:105640002807000E3D49C8703B480088000A0871D1
:1056500039480078487132E001253C48007800F074
:105660000F0020B1012808D002281CD110E03248D8
:10567000406820433049486015E02F484068012CBD
:1056800001DA012100E0002108432B4948600AE0CB
:1056900029484068022C01DA012100E0002108437A
:1056A0002549486000BF00BF2807000E2349C87085
:1056B00021488088000A08711F48007948712448F1
:1056C00001681E48FFF72EFE214801681B4800F0C4
:1056D0004FFE70BD10B5184890F844001749087087
:1056E000154890F848004870134890F840008870BA
:1056F0001648007800F0100048B90020C8700E4825
:105700000088000A08710C480078487109E01020F0
:105710000A49C87008488088000A0871064800795C
:1057200048710B4801680548FFF7FCFD084801680F
:10573000024800F01DFE10BD34C4072058190010A7
:1057400000C0092000005307BC19001044010010DC
:10575000400100102DE9F0478548407984490979D6
:1057600040EA012400BF204602F0C6FA8246814882
:105770000168504602F0ECFA814602F0F3F9074660
:105780007D4A7E4B01F098FD054601F063FD7C49A2
:1057900008600846006802F08FFA7A498861BDE81F
:1057A000F08700207849096CB0291FD006DC0A294F
:1057B00010D0992909D0A52927D10DE0D8291AD0D0
:1057C000D9291DD0DD2920D10BE0062008216F4A00
:1057D00011601AE0082018E0062008216B4A1160C9
:1057E00013E006202C21694A11600EE006200821F2
:1057F000664A116009E006200821644A116004E04D
:1058000006200821614A116000BF00BF704710B533
:10581000DD205D4948640846B0F8580080B28865CC
:10582000534800F0CCFE5A49086008460068012839
:1058300013D14F480078CC280ED04D4800F04BFED5
:105840005148806D00F580704F498865084690F892
:105850005800474981F8630088E04D4800680228F5
:105860000ED1434840784849896C88427ED04048F0
:1058700000F031FE4448806D401C4349886575E066
:1058800043480068032808D1394880783E490864B5
:10589000FFF787FF3F49086068E03D48006804283B
:1058A00008D13C480068062804D13148C0783A49FC
:1058B00008605BE03648006805280CD13548006870
:1058C000072808D12A48C078334908602848007959
:1058D000324908604AE02E480068062810D12D4859
:1058E000006808280CD12248C0782B49086020485D
:1058F00000792A4908601E4840792949086035E046
:1059000024480068401E2249096888422ED218485F
:1059100000F0E1FD1E4801681548FFF703FD28B3BC
:105920001948006CD8280DD004DC0A2810D099281A
:105930001BD104E0D92808D0DD2816D111E0FFF7EB
:1059400018FD12E0FFF71BFE00BFFFF7C3FE0CE0DF
:1059500013480268114801680F480068FFF7FAFE13
:1059600003E001200F49086000BF00BF10BD000028
:105970005819001074C10720560E2DB26D44C64050
:1059800070C10720BC19001034C40720400100106A
:10599000300100103C0100104401001048010010CB
:1059A0004C01001024010010F949096841F0100170
:1059B000F74A11601146096841F0400111608321E6
:1059C000F44AD160F4490968F44A92FBF1F188B2D3
:1059D0000146C21700EB12621212EE4B5A60C21758
:1059E00000EB12621212A0EB02221A6003211A4687
:1059F000D160072191607047E549096941F00201D2
:105A0000E34A11611146096941F0080111618321DE
:105A1000E34AD160E3490968E04A92FBF1F188B2B8
:105A20000146C21700EB12621212DD4B5A60C21718
:105A300000EB12621212A0EB02221A6003211A4636
:105A4000D160072191607047D149096841F4801104
:105A5000CF4A11601146096841F480011160D249B2
:105A6000096841F08071D04AC43AC2F8C410832159
:105A7000CE4AD160A2200146C21700EB1262121278
:105A8000CA4B5A60C21700EB12621212A0EB02223C
:105A90001A6003211A46D160072191607047BC4902
:105AA000496841F44021BA4A51601146496841F4BD
:105AB00040115160BC49096841F00071BA4AC43ACA
:105AC000C2F8C4108321BA4AD160BA490968B34AFE
:105AD00092FBF1F188B20146C21700EB126212127A
:105AE000B34B5A60C21700EB12621212A0EB0222F3
:105AF0001A60B14909681A46D16007219160704760
:105B000030B502460B46A249096841F48011A04C09
:105B100021602146096841F480012160A249096899
:105B200041F08071A04CC43CC4F8C41083219F4C48
:105B3000E1609A49B1FBF2F188B20146C41700EB6B
:105B400014642412994D6C60C41700EB1464241281
:105B5000A0EB04242C602946CB6007212C46A160D1
:105B600030BD30B502460B468949496841F44021B1
:105B7000874C61602146496841F4401161608A495F
:105B8000096841F00071884CC43CC4F8C4108321FA
:105B9000874CE1608149B1FBF2F188B20146C4173C
:105BA00000EB14642412824D6C60C41700EB146483
:105BB0002412A0EB04242C602946CB6007212C463C
:105BC000A16030BD70B503460C467C49B1FBF4F1D1
:105BD000491C88B203BB6E49096841F010016C4D45
:105BE00029602946096841F0400129608321694DF7
:105BF000E9600146C51700EB15652D12654E75600D
:105C0000C51700EB15652D12A0EB05253560314653
:105C1000CA6007213546A960012B20D15C4909697A
:105C200041F002015A4D29612946096941F00801F4
:105C3000296183215A4DE9600146C51700EB1565BE
:105C40002D12574E7560C51700EB15652D12A0EB90
:105C5000052535603146CA6007213546A960022B0B
:105C600028D14B49096841F48011494D29602946E2
:105C7000096841F4800129604B49096841F080714D
:105C8000494DC43DC5F8C4108321484DE960014623
:105C9000C51700EB15652D12444E7560C51700EB56
:105CA00015652D12A0EB052535603146CA60072128
:105CB0003546A960032B28D13549496841F4402174
:105CC000334D69602946496841F44011696036499D
:105CD000096841F00071344DC43DC5F8C4108321FA
:105CE000334DE9600146C51700EB15652D12304EA6
:105CF0007560C51700EB15652D12A0EB0525356005
:105D00003146CA6007213546A96070BD00BF2149F0
:105D1000496901F020010029F9D01E490860704747
:105D200000BF1C48406900F001000028F9D0194864
:105D30000068704700BF1A48406900F00100002861
:105D4000F9D017480068704700BF1848406900F054
:105D500001000028F9D015480068704700BF1448BA
:105D6000406900F001000028F9D011480068704730
:105D70000848406900F0010008B101207047002088
:105D8000FCE70748406900F00100C8B101207047F6
:105D900000C0024000C00040B0C3072084D71700F5
:105DA00000000140B4C30720C4C00F400080094078
:105DB00000C00940BCC30720C0C30720105E5F00BD
:105DC00000207047FA48406900F0010008B1012046
:105DD00070470020FCE7F748406900F0010008B177
:105DE000012070470020FCE700B5024603E012F8EE
:105DF000010BFFF78BFF10780028F8D100BD00BF22
:105E0000EB49496901F020010029F9D0E84908600F
:105E100070471CB502460A2092FBF0F100FB1120EE
:105E2000303080B2ADF806000A2092FBF0F00A2173
:105E300090FBF1F401FB1400303080B2ADF80400A7
:105E40000A2092FBF0F090FBF1F090FBF1F401FBE3
:105E50001400303080B2ADF802000A2092FBF0F05E
:105E600090FBF1F090FBF1F090FBF1F401FB1400DA
:105E7000303080B2ADF80000002305E03DF813009B
:105E8000FFF744FF581CC3B2042BF7DB1CBD70475F
:105E900000B5C948006800F0005050B10A20FFF773
:105EA000F6FFC548006820F00050C3499439C1F896
:105EB000940000BD00B5C048006800F0005050B923
:105EC000BD48006840F00050BB499439C1F89400C7
:105ED0000A20FFF7DCFF00BD00B5B8480068E0B954
:105EE000B7480068B7490968884216D0B648406983
:105EF00000F0200088B1B3480068401CB149086038
:105F000008460088C0F309000860FFF7D3FFAF48D8
:105F1000AC490968405CAC490860AB48406900F096
:105F2000010078B1AA480068401CA94908600846E9
:105F30000088C0F309000860A3480068A549A44A86
:105F400012688854A048406900F0400010B9FFF77B
:105F5000B1FF01E0FFF79CFF00BD9F480068C8B992
:105F60009E4800689E490968884213D09D48406950
:105F700000F0200070B19A480068401C9849086001
:105F800008460088C0F30900086097480968405C2B
:105F9000944908609348406900F0010078B1934843
:105FA0000068401C9149086008460088C0F3090059
:105FB00008608C4800688E498C4A12688854704783
:105FC00000B57D489438406D00F0040050B10A20BF
:105FD000FFF75DFF78489438406D20F00400764963
:105FE0009439486500BD00B573489438406D00F0A1
:105FF000040050B970489438406D40F004006E4978
:10600000943948650A20FFF742FF00BD00B5724889
:106010000068F0B911E072480068401C70490860DF
:1060200008460088C0F309000860FFF7DCFF6E48EF
:106030006B490968405C6B490860684800686849BA
:106040000968884205D06748406900F020000028B0
:10605000E1D10FE065480068401C644908600846CB
:106060000088C0F3090008605E48006860495F4A24
:10607000126888545B48406900F001000028E9D1AB
:106080005848406900F0400010B9FFF7ACFF01E04C
:10609000FFF796FF00BD00B547489438406D00F407
:1060A000005050B10A20FFF7F2FE43489438406D8B
:1060B00020F4005040499439486500BD00B53E4881
:1060C0009438406D00F4005050B93B489438406D0E
:1060D00040F400503849943948650A20FFF7D7FE4C
:1060E00000BD00B543480068E0B943480068434933
:1060F0000968884216D02E48406900F0200088B117
:106100003E480068401C3D49086008460088C0F3CE
:1061100009000860FFF7D2FF394838490968405C38
:10612000234908602248406900F0010078B13548F1
:106130000068401C3349086008460088C0F3090025
:1061400008601B48006830492E4A12688854184875
:10615000406900F0400010B9FFF7B0FF01E0FFF721
:106160009AFF00BD00B514489438406900F0807073
:1061700050B10A20FFF78BFE0F489438406920F099
:1061800080700D499439486100BD00B50A489438C3
:10619000406900F0807050B907489438406940F079
:1061A00080700549943948610A20FFF770FE00BDF0
:1061B0000080094000C0094094C0092024C4072081
:1061C000CCC30720D0C3072000C00040DC3500103E
:1061D000C8C30720DC31001028C40720DCC3072017
:1061E000E0C3072000000140DC3D0010D8C30720B9
:1061F000DC3900102CC40720ECC30720F0C30720B3
:10620000DC450010E8C30720DC41001000B5F6486B
:106210000068E0B9F5480068F5490968884216D079
:10622000F448406900F0200088B1F1480068401C43
:10623000EF49086008460088C0F309000860FFF7CE
:10624000A4FFED48EA490968405CEA490860E9486A
:10625000406900F0010078B1E8480068401CE74957
:10626000086008460088C0F309000860E14800683B
:10627000E349E24A12688854DE48406900F0400071
:1062800010B9FFF782FF01E0FFF76CFF00BD00B51A
:10629000DC480068E0B9DC480068DC4909688842ED
:1062A00016D0DB48406900F0200088B1D94800686A
:1062B000401CD849086008460088C0F309000860FF
:1062C000FFF7FCFED448D3490968405CD049086018
:1062D000CF48406900F0010078B1D0480068401C08
:1062E000CE49086008460088C0F309000860C84825
:1062F0000068CB49C94A12688854C548406900F013
:10630000400010B9FFF7DAFE01E0FFF7C4FE00BD60
:106310000021C44A11600FE0C3490968491CC24A00
:10632000116011460988C1F30901116010F8011BC1
:10633000BE4ABD4B1B68D15401780029ECD170478F
:106340000021BB4A11600FE0BA490968491CB94AEB
:10635000116011460988C1F30901116010F8011B91
:10636000B54AB44B1B68D15401780029ECD1704771
:1063700010B50022AB4B1A6010E0491EAA4A126801
:10638000521CA94B1A601A461288C2F309021A60FD
:1063900010F8012BA54BA44C24681A550029ECD108
:1063A00010BD0021974A11600FE0A4490968491CFB
:1063B000A24A116011460988C1F30901116010F861
:1063C000011B954A9D4B1B68D15401780029ECD1E3
:1063D00070470021844A11600FE084490968491C14
:1063E000824A116011460988C1F30901116010F851
:1063F000011B814A7D4B1B68D15401780029ECD1E7
:10640000704730B505460C4614B92846FFF780FFA3
:10641000012C02D12846FFF793FF022C02D1284617
:10642000FFF7BFFF022C02D12846FFF7D2FF30BD95
:106430007D490968491C7C4A116011460988C1F3ED
:1064400009011160794A784B1B68D054704779492B
:106450000968491C774A116011460988C1F309018E
:106460001160754A734B1B68D054704773490968B3
:10647000491C724A116011460988C1F30901116073
:10648000654A6E4B1B68D054704758490968491CCF
:10649000564A116011460988C1F309011160564A34
:1064A000524B1B68D054704730B505460C4614B9A2
:1064B0002846FFF7BDFF012C02D12846FFF7C7FF92
:1064C000022C02D12846FFF7D1FF032C02D1284627
:1064D000FFF7DBFF30BD014600200FE0401C584AAB
:1064E0001268521C564B1A601A461288C2F30902EF
:1064F0001A60544A1B68D25C01F8012B504A12689A
:10650000514B1B689A42E9D1002201F8012B7047D8
:10651000014600200FE0401C4C4A1268521C4B4BB5
:106520001A601A461288C2F309021A60484A1B68A8
:10653000D25C01F8012B454A1268464B1B689A420F
:10654000E9D1002201F8012B7047014600200FE03D
:10655000401C414A1268521C3F4B1A601A4612886E
:10656000C2F309021A602E4A1B68D25C01F8012BA3
:10657000394A1268294B1B689A42E9D1002201F876
:10658000012B7047014600200FE0401C334A12687F
:10659000521C324B1A601A461288C2F309021A6062
:1065A000174A1B68D25C01F8012B2C4A1268134B66
:1065B0001B689A42E9D1002201F8012B704701467D
:1065C00000201F4B1A6807E0401C521CC2F309024E
:1065D0001C4B9B5C01F8013B1B4B1B689A42F3D19F
:1065E000002301F8013B704730C40720FCC307209B
:1065F00000C4072000C00940DC4D0010F8C307208C
:10660000DC4900102CC407200CC4072010C407204C
:1066100000800940F0C30720DC450010E8C30720D4
:10662000DC41001024C40720CCC30720DC35001057
:1066300028C40720DCC30720DC3D0010ECC3072082
:10664000C4C30720DC310010C8C30720D4C307200F
:10665000DC390010D8C30720E4C30720F4C30720A7
:1066600001460020444B1A6807E0401C521CC2F34C
:106670000902424B9B5C01F8013B414B1B689A426B
:10668000F3D1002301F8013B7047014600203D4B48
:106690001A6807E0401C521CC2F309023A4B9B5C8B
:1066A00001F8013B394B1B689A42F3D1002301F8F2
:1066B000013B704701460020354B1A6807E0401C3B
:1066C000521CC2F30902334B9B5C01F8013B324B75
:1066D0001B689A42F3D1002301F8013B70472F4811
:1066E00000682F490968884201D0012070470020C6
:1066F000FCE72148006822490968884201D001204E
:1067000070470020FCE71F4800682049096888425C
:1067100001D0012070470020FCE71D4800681E4999
:106720000968884201D0012070470020FCE71D481D
:10673000406900F0400008B9012070470020FCE7E4
:106740001948406900F0400008B901207047002056
:10675000FCE71648406900F0400008B90120704786
:106760000020FCE71248406900F0400008B9012011
:1067700070470020FCE70000D4C30720DC3900107C
:10678000D8C30720E4C30720DC410010E8C307207A
:10679000F4C30720DC490010F8C30720C4C3072056
:1067A000C8C3072000C0004000000140008009402D
:1067B00000C0094010B54C1084EA530404D540428F
:1067C000C1F1000138BF491E1B4204D55242C3F13A
:1067D000000338BF5B1E00F077F814F0804F04D040
:1067E0004042C1F1000138BF491E14F0004F04D0EF
:1067F0005242C3F1000338BF5B1E10BD0B4910B5F8
:10680000A1F17C020A4CC2E93712372106E000EB05
:10681000104342F82130074B00FB03400B1EA1F14F
:106820000101F4DC10BD0120E8E70000D4F20720EC
:10683000E119D666CD0D0100032A40F2308010F038
:10684000030C00F0158011F8013BBCF1020F62440B
:1068500098BF11F801CB00F8013B38BF11F8013B9C
:10686000A2F1040298BF00F801CB38BF00F8013B49
:1068700011F0030300F0AA80083AC0F0088051F834
:10688000043B083A51F804CBA0E80810F5E7121DC4
:106890005CBF51F8043B40F8043BAFF30080D207E3
:1068A00024BF11F8013B11F801CB48BF11F8012BAF
:1068B00024BF00F8013B00F801CB48BF00F8012BD2
:1068C000704770477047704753EA020C00F06980C8
:1068D0002DE9F04B4FF00006002B1FBFB3FA83F5F4
:1068E00003FA05F424FA05F65E4012BF1643B2FA25
:1068F00082F502FA05F4C5F120051EBF22FA05FC57
:1069000044EA0C04203556EA044C4FEA144418BFFC
:10691000641C4FF000084FF00009904271EB030C2B
:1069200039D3002919BFB1FA81F701FA07F6B0FA95
:1069300080F700FA07F6C7F120071EBF20FA07FC10
:1069400046EA0C062037B6FBF4FCA7EB0507103F20
:1069500007F01F0BCBF120060CFA0BFB2CFA06F606
:1069600044BFB3460026202FA4BF5E464FF0000B65
:106970005BEA060C08BF4FF0010B19EB0B09ABFBF0
:10698000027C48EB0608C01B06FB02CC0BFB03CCC9
:1069900071EB0C01C1E70B46024641464846BDE893
:1069A000F08B13B54FF000004FF00001AFF3008003
:1069B000BDE81C40704710B500F03AF8006810BD03
:1069C00010B5044600F034F8046010BD10B5203A4C
:1069D000C0F00B80B1E81850203AA0E81850B1E898
:1069E0001850A0E81850BFF4F5AF5FEA027C24BF4E
:1069F000B1E81850A0E8185044BF18C918C0BDE845
:106A000010405FEA827C24BF51F8043B40F8043B0D
:106A100008BF7047D20728BF31F8023B48BF11F8C2
:106A2000012B28BF20F8023B48BF00F8012B70471C
:106A300000487047DC52001000487047DC520010DC
:106A40007546FFF7F9FFAE4605006946534620F04C
:106A50000700854618B020B5F9F7CCFBBDE820400B
:106A60004FF000064FF000074FF000084FF0000B0A
:106A700021F00701AC46ACE8C009ACE8C009ACE8BD
:106A8000C009ACE8C0098D4670470446AFF30080EA
:106A90002046F9F780FB704701491820ABBEFEE79E
:106AA0002600020002461068884200D91160704733
:106AB000490050EAC12018BF04204A0D18BF40F019
:106AC000010040F2FF72B2EB515F08BF40F00200DC
:106AD000012808BF052070472DE9F74F144694B0F0
:106AE0000021C4E902111599079121F00045C94917
:106AF0008D4206DC1599C4E9000117B00020BDE8FD
:106B0000F08FC549DFF814A3A9423CDD0799C44EB4
:106B10000029C44FC44A1599534619DD00F038FFC7
:106B2000554506D0C14AC24B00F032FFC4E900010E
:106B30000AE04FF0D352BE4B00F02AFF32463B46EC
:106B400000F026FFC4E9000117B00120BDE8F08F76
:106B500000F0B2FB554506D0B44AB54B00F0ACFB93
:106B6000C4E900010AE04FF0D352B14B00F0A4FB9E
:106B700032463B4600F0A0FBC4E9000117B04FF0DD
:106B8000FF30BDE8F08FAB49A942159978DB21F0C1
:106B9000004183468846A84AA84B00F0EFFD00223A
:106BA000A74B00F089FB00F08FFD099000F0BBFDC2
:106BB00006460F469C4A534600F0E0FD43465A46BF
:106BC00000F0DAFE80468A46984A994B30463946AC
:106BD00000F0D4FD2A0D01250B924246534600F0E9
:106BE000CBFE032DC4E9000139D00B98C1F30A5143
:106BF000401A05EB45111139814230DA9148C346FC
:106C0000784400EB0510CDF80CA00C90D0E90023DF
:106C10003046394600F0B2FD02460B46049106901C
:106C20005846039900F0B4FE80468A4602460B4659
:106C30005846039900F0ACFE049B069A00F0A8FEAB
:106C400083460C9803913946D0E90223304600F080
:106C500095FD5A46039B00F09BFE6D1CBDE707980F
:106C60000028A2BF099817B0BDE8F08F616881F0D5
:106C700000416160099817B04042BDE8F08FFFE71E
:106C800084461598C1F31301C0F30A50A0F2F53001
:106C90004FEA601800F01F06C6F120001390002094
:106CA0000690079041F4801E05206D4676B1664A35
:106CB00008EB00017A4452F8213002EB8101B34025
:106CC0004A68139922FA01F1194305E05F4908EB7C
:106CD0000002794451F82210A1FB0E27A1FB0C13EE
:106CE0001A449A4234BF0123002303EB070A05EB41
:106CF0008003D3E901B70F448F4234BF0121002143
:106D000093448B4411B1934502D903E0934501D2DA
:106D1000012100E00021C3E901B7514445F82010EA
:106D2000011EA0F10100C1DC0298059F00F1005096
:106D3000800F12900298DDE90356800000F0F3FC0A
:106D4000834628460D9100F005FD6FF01D0201F00D
:106D50007CF9CDE90E01304600F0FCFC6FF03D02FD
:106D600001F073F980468A46384600F0F3FC6FF074
:106D70005D0201F06AF9074642465346119100F060
:106D80009BFADDE90E2300F097FA5A460D9B00F0BE
:106D900093FA00250E465A4628460D9B00F0F8FD52
:106DA000DDE90E2300F0F4FD4246534600F0F0FD0D
:106DB0003A46119B00F0E0FDDFF898A0244A5346C4
:106DC00000F0DCFC07468846234A244B314628461F
:106DD00000F0D4FC3A46434600F06EFA0746884677
:106DE0004FF0A84253463146284600F0C7FC3A46C9
:106DF000434600F061FA159A12F0004F04D0129A3F
:106E000081F0004152421292C4E90001129817B079
:106E1000BDE8F08FFB21E93F7CD90240FB21F93F1F
:106E20007370032E8A19A33B000040543163621A29
:106E300061B4D03DFB21394183C8C96D305FE43F67
:106E40000000E03F04150000801400006214000000
:106E5000182D4454FB21F93D3326A611460B113C55
:106E60002DE9FF4D21F0004807460C46B8F1795F47
:106E700008DA00F029FC002801BF0020324904B0E4
:106E8000BDE8F08D3A4623461046194600F076FCE0
:106E9000054602462D480E460B460621784400F072
:106EA0005DF82A46334600F069FCDDE9022382469C
:106EB0008B463846214600F061FC04460F46524698
:106EC0005B462846314600F059FC22463B4600F01E
:106ED0005FFD07468A464FF0FF322846314601F0F3
:106EE000B4F81B4A90450ADA3A46534600F050FD82
:106EF00004B00022BDE8F04D134B00F03DBD154A33
:106F00004245A8BFA8F500154FF00004B8BF124DC8
:106F100022462B4600F03CFD0646884622462B467C
:106F20000020094900F034FD04460D463A46534618
:106F30003046414600F02CFD04B022462B46BDE809
:106F4000F04D00F019BD00000000F03F38120000C5
:106F50003333D33F0000E93F0000D23F2DE9F04139
:106F60004F1E00EBC7010446D1E9000115461E463D
:106F700037F006020DD02A46334600F0FFFB7F1E95
:106F800004EBC703D3E9002300F096F937F00602BB
:106F9000F1D1022F25D0042F13D0062F18BFBDE842
:106FA000F0812A46334600F0E9FBD4E90A2300F0D9
:106FB00083F92A46334600F0E1FBD4E9082300F0C8
:106FC0007BF92A46334600F0D9FBD4E9062300F0CA
:106FD00073F92A46334600F0D1FBD4E9042300F0CC
:106FE0006BF92A46334600F0C9FBD4E9022300F0CE
:106FF00063F92A46334600F0C1FBD4E90023BDE81B
:10700000F04100F059B900002DE9FF4D054621F08F
:10701000004084B00C46B0F1795F0BDA2846FFF7E8
:1070200047FD042808BF00F06FF8284608B0214645
:10703000BDE8F08D2A460B46104600F09FFB064641
:107040000F462A46234600F099FB804626488A468A
:1070500032463B4605217844FFF780FF834610986F
:10706000029160B3214A224B4046514600F086FB14
:10707000CDE900015A4640465146029B00F07EFB96
:1070800082468846DDE906014FF0FF3200F0DDFF61
:107090005246434600F07CFC32463B4600F06EFB15
:1070A000DDE9062300F074FCDDE9002300F070FC4C
:1070B00008B02A462346BDE8F04D00F05DBC0B4603
:1070C0005A463046394600F059FB084A084B00F052
:1070D000F3F84246534600F051FB08B02A462346D7
:1070E000BDE8F04D00F0E8B876110000495555555F
:1070F0005555C5BF012200F0A8BF00221346104617
:10710000114600F089B90000024A0020110700F082
:107110009CBF000001FDFFFF00B5244B21F00042A1
:1071200087B09A42DCBF0022134629DD204B9A42E9
:1071300008D140B94FF00100FFF742FCFFF7DDFF37
:1071400007B000BD03DBFFF7D5FF07B000BD02AA03
:10715000FFF7C2FC10F0030104BF0DF1080C9CE81E
:107160000F000DD0012001290ED0022914D00DF1FD
:10717000080C00909CE80F00FFF746FF07B000BD29
:10718000FFF76EFE07B000BD0DF1080C00909CE803
:107190000F00FFF739FF05E00DF1080C9CE80F0028
:1071A000FFF75EFE07B081F0004100BDFB21E93F23
:1071B0000000F07F00B5254B21F0004287B09A42D5
:1071C00003DC0022134600922BE0214B9A4208D1A7
:1071D00040B94FF00100FFF7F3FBFFF78EFF07B058
:1071E00000BD03DBFFF786FF07B000BD02AAFFF773
:1071F00073FC10F003014FF001000DD0012914D0F1
:1072000002291AD00DF1080C9CE80F00FFF728FEA8
:1072100007B081F0004100BD0DF1080C00909CE822
:107220000F00FFF7F1FE07B000BD0DF1080C9CE860
:107230000F00FFF715FE07B000BD0DF1080C009020
:107240009CE80F00FFF7E0FEE2E70000FB21E93FCA
:107250000000F07F21F00042A2F16052B2F5801FE1
:1072600001F0004328BFD2F17F6C0BD95FEA001C0C
:1072700043EAC20242EB507018BF704728BF20F0AB
:1072800001007047B2F5801FBCBF184670474FEA37
:10729000410C1CF5001F02D2084600F020BE70B55C
:1072A00000F016FB00000089FFF7F6BF4FF000402A
:1072B000A0F580007047000010B591EA030F48BFA9
:1072C00083F0004300F16C83841A71EB030C05D248
:1072D000121943EB0C03001B61EB0C01DFF824E1F6
:1072E0004FEA1154A4EB135C1EEA430F18BF9EEA49
:1072F000445F73D023EA0E03DCF1200E21EA04512F
:1073000043F4801332D322FA0CFE10EB0E0023FA62
:107310000CFE41EB0E01CCF1200E03FA0EFE10EB39
:107320000E0051F10001B1F5801FCCF1200E32D2D8
:1073300001EB045112FA0EF2BDE8104058BF70473D
:10734000401C38BF5FEA420218BF7047002814BFD4
:1073500020F0010041F100014FEA410313F5001F45
:1073600038BF7047A1F1C04100F000BB012A43EBD8
:107370000302ACF1200CDCF11F0E32BF4FF0000E07
:1073800023FA0CF310EB030041EB0451B4EB115F53
:10739000D0D0A1EB045101F5801149085FEA30001B
:1073A00001EB04510ED350F1000038BF12FA0EFE6B
:1073B00008D1BDE81040C9E7401C38BF5FEA42026F
:1073C000CAD1C3E7BDE810404FEA410313F5001FDF
:1073D00038BF7047A1F1C04100F0C8BA9EEA445FCF
:1073E00008D011EA5E0FBDE8104004BF01F0004173
:1073F00000207047BDE8104070B500F069FA00BF8A
:1074000064FBBE3E0000E0FF02494FF0000000F0C8
:10741000EABD00BF0000F87F2DE9C04130B4DFF8BD
:10742000A0C23CEA111418BF3CEA131400F0EC802F
:1074300081EA03051CEA111444EAD57418BF1CEA5A
:10744000131500F0C780A4EB05044FF0004545EA92
:10745000C12145EAC32341EA505143EA525304F1A2
:107460007F74994204F500344FEAC0204FEAC222EB
:1074700008BF904200F09C804FEA13650FF240165F
:10748000765D4FEA134506FB05F7C7F1807706FBEB
:1074900007F74FEAD737A7FB03687642C8F580386D
:1074A000A7FB06CE38BFA8F1010807FB08E64FF09E
:1074B000000EA6FB028CE6FB03CEDCF1000CCEF145
:1074C000004E38BFAEF1010EA6FB0C584FF000077E
:1074D0004FF00005E6FB0E87A1FB08C6A0FB07CE18
:1074E00016EB0E0645F10005E1FB076515F1E04ED0
:1074F0007EBFA4F580345FEA46066D4116F1800731
:1075000045F100054FEA17274FEA066647EA056787
:10751000A6F1DE46B6F1805F4FEA15251FD9384641
:1075200024F0010C05EBC471BCF1FE6F01EB0C11F2
:1075300002D8F0BCBDE8008124425CBF01F5801E8A
:107540009EEAC47F02D4F0BCBDE80081244238D456
:10755000F0BCA1F1C041BDE8004100F007BA4FEA1C
:10756000D22242EA43524FEAD323A7FB02864FEAD4
:10757000D02040EA415007FB03661EEA0E0F4FEA97
:10758000D12105FB026658BFA6EB0056B6EB0056AC
:107590004FEA520E4EEAC37E18EB0E0E56EB530E18
:1075A000BDD518EB02085E417F1C55F10005B6E71A
:1075B0004FF480154FF000074FF000064FF0000821
:1075C000ADE7F0BC4FF0000001F1C04101F0004117
:1075D000BDE8008111EA0C1F0CEA131500D00CE085
:1075E00013EA0C1F00F025804FF00000F0BC81EA88
:1075F000030101F00041BDE80081F0BCBDE800419D
:1076000081EA030100F0B2B9F0BCBDE8004170B5F9
:1076100000F05EF9097EFC3E00F007B881EA030144
:107620004FF0000001F00041704781EA030100F0D3
:107630009DB9F0BCBDE800414FF000002149704702
:10764000FFFDFBF9F7F5F4F2F0EEEDEBE9E8E6E427
:10765000E3E1E0DEDDDBDAD8D7D5D4D3D1D0CFCDAE
:10766000CCCBCAC8C7C6C5C4C2C1C0BFBEBDBCBBE7
:10767000BAB9B8B7B6B5B4B3B2B1B0AFAEADACABE2
:10768000AAA9A8A8A7A6A5A4A3A3A2A1A09F9F9EBC
:107690009D9C9C9B9A99999897979695959493936E
:1076A000929191908F8F8E8E8D8C8C8B8B8A898905
:1076B0008888878786858584848383828281818088
:1076C0000000FF070000F87F4FEA41034FEA5353E1
:1076D000A3F58063D3F11E03C8BFD3F1210C0CDDE9
:1076E0004FF0004242EAC12242EA505232FA03FC11
:1076F0008CEAE17CACEBE1707047102BC4BF00203A
:10770000704703F5787CBCF1FF3F04D06FF0004276
:1077100082EA2100704770B500F0DAF849922480BF
:1077200000207047F2E710F0004248BF4042B0FA34
:1077300080F310FA03F10AD0C3F11D0303F580634F
:107740004FEA415002EB035202EBD12170474FF058
:1077500000007047B0FA80F310FA03F10AD0C3F1C9
:107760001D0303F580634FEA41504FEA035202EBD9
:10777000D12170474FF0000070470000DFF848C18A
:1077800070B51CEA111E1EBF1CEA13159EEA0C0FF1
:1077900095EA0C0F00F06F8081EA030423EA4C1392
:1077A0004EEAD47E21EA4C1141F4801143F4801357
:1077B000AE44A1FB024CA0FB0365AEF17F7E3619FF
:1077C00055EB0C05A1FB034C4CF10003A0FB021C84
:1077D00016EB0C06654153F10003094218BF46F051
:1077E000010613F4007F0BD14FEA03314FEA053055
:1077F000340341EA155140EA16506FF003020AE0E3
:107800004FEAC3214FEAC520F40241EA555140EA4C
:1078100056506FF0020202EB2E4201EB025585EA50
:10782000CE710AD05FEA440C18BF24F0004450F136
:10783000000041F1000120EAD47040F2FE7C624574
:1078400000D270BDA84214BF4FF080444FF04044B6
:10785000002E08BF0024BEF1806FA8BFA1F1C04177
:10786000BDE8704080F282804FF0000001F1C0411D
:1078700001F0004170479EEA0C0F0CEA131518BF87
:1078800095EA0C0F06D04FF0000081EA030E0EF0CF
:10789000004170BD00F01CF88900013E00F007B8FF
:1078A00000F009B84FEA430C5FEA5C5C08D081EA5B
:1078B000030100F05BB84FEA410C5FEA5C5CF6D173
:1078C0004FF00000014970470000FF070000F87FFB
:1078D0000EF1020E2EF0030E5EF8046B364205D454
:1078E000012A43EB030515F5001F12D8012841EBCF
:1078F000010C1CF5001F0CD80ED14FEAD17C15F5F8
:10790000001F0CEB4C0C0CF1020C08BF4CEBD37CB1
:1079100004E04FF0080C01E04FEAD37C0CEB4C057F
:1079200026FA05F606F00706B6F1040C06D20EEBB1
:10793000860CBDE870404CF0010C6047DFE80CF0AD
:10794000090B02024FF000414FF00000A1F50021A9
:1079500070BD19461046012851EB010418BFD4F53B
:10796000001484BF002001F0004170BD0808A0F59C
:1079700000114FEA3101704791EA030F10B581F011
:1079800000413FF5A1AC83F0004300F009B80000CE
:1079900010B591EA030F48BF83F000433FF594AC64
:1079A000841A71EB030C07D212198CF0004C43EBD4
:1079B0000C03001B61EB0C01DFF8A4E14FEA11544A
:1079C000A4EB135C1EEA430F18BF9EEA445F00F06D
:1079D000B08023EA6E03524221EA0451C3EB6E03E6
:1079E00038BF5B1EDCF1200E25D322FA0CFE10EB13
:1079F0000E0043FA0CFE41EB0E01CCF1200E03FA0F
:107A00000EFE10EB0E0051F10001CCF1200E29D436
:107A100012FA0EF201EB0451BDE8104058BF704756
:107A2000401C1CBFB2F1004F704700280CBF491C1E
:107A300020F00100704712EB020E43EB030218BF67
:107A40004FF0010E4EEA4202ACF1200CDCF11E0EAA
:107A500054D943FA0CFE10EB0E0051F1FF31CCF17A
:107A60001E0ED5D50EF1010E12FA0EFE404141EB6D
:107A7000010101EB445C5FEA5C5C10D910EBDE7045
:107A800001EB045138BFBEF1004FBDE8104018BFF4
:107A9000704700280CBF491C20F00100704730D20D
:107AA0004FEAD42C11F5001124F400641BD0B1FA74
:107AB00081F20B3AA41AA41ED2F12003914030FAAD
:107AC00003F31943904001EBCC71002C01EB0451FE
:107AD000BDE81040A8BF704701F1C0414FF0000061
:107AE00001F000417047B0FA80F310FA03F100D1C1
:107AF00010BDE41A173C4805C90AE4E701EB04513C
:107B000010BD491001EB0451BDE810404FEA3000B0
:107B100002E04FF0000170474A0008BF0042F8D071
:107B2000B2F5001F28BF704701F000414FF0000080
:107B300070479EEA445F07D011EA5E0FBDE810402F
:107B400004BF002100207047BDE8104070B5FFF76A
:107B5000BFFE00BF40DFF63E83F000411046704795
:107B60000000E0FF43004FEAD30C4FEA3C0C4340D7
:107B70001FBF40070CF1605113F0FE4F70471CF01F
:107B8000006F03D100200CF0004170470CF000435F
:107B900043EA507010B540EACC0000F05AF900BF3B
:107BA000000000924FEA0001FFF7E0BE4FF00041F5
:107BB0004FF00000A1F500217047000090EA010F8E
:107BC00048BF81F0004100F1A081421A3CBF801AF9
:107BD00089184FEAD0524FF07F4C1CEA410FA2EBBC
:107BE000D15318BF9CEA026F00F03B804FF0004C6D
:107BF0004CEA00204CEA012121FA03FC10EB0C0CAA
:107C00001ED202F1FF325FEA1C2040EBC25038BFA7
:107C100070471CF07F0F4FEA400C18BFBCF17F4F3C
:107C200038BF7047C3F12003994008BF20F001001E
:107C3000BCF17F4F38BF7047A0F1C04000F04FB992
:107C40004FEA3C00000A40EBC25028BF1CF0FF0F77
:107C50004FEA400CE6D018BFBCF17F4F38BF7047E9
:107C6000EAE79CEA026F05D010EA5C0F08BF00F05B
:107C70000040704710B500F0ECF800BF64FBBE3E5A
:107C800041000B0ED3F19E0208D950F400034FEAD5
:107C9000032323FA02F048BF4042704710B500F0BA
:107CA000D8F800BF49922480002070476FF000424E
:107CB00082EA200070470000C10DD1F19E0206DB70
:107CC0004FEA002343F0004323FA02F070470042DA
:107CD00007D54FEA4001B1F1FE4F02D24FF000004C
:107CE000704710B500F0B5F8499224800020704725
:107CF0006FEA20007047000010F0004148BF40428A
:107D0000B0FA80F310FA03F2C3F19D030BD051EAED
:107D1000C35101EB1220530638BF704700F1010038
:107D200008BF20F001007047B0FA80F310FA03F2A8
:107D3000C3F19D030AD0D90501EB1220530638BFC9
:107D4000704700F1010008BF20F0010070470000FB
:107D50004FF47F0C1CEAD0121EBF1CEAD11392EA2A
:107D60000C0F93EA0C0F00F0478090EA010F48BF18
:107D700042F480724FF0004C4CEA00204CEA0121A2
:107D800002EB0302A0FB0113A2F50002002918BFB9
:107D900043F001035B0028BF4FEA330342EB22426A
:107DA0005FEA132C4CEBC2502EBFBCEB436FB2F515
:107DB0007C0F70474FEA036CBCF1004F08BF20F006
:107DC0000100B2F57C0F38BF70470BD582F0FF027F
:107DD00012F5803FC8BF704700F1C040D8BF00F027
:107DE0000040704700F5000C5FEA4C0C48BF70473C
:107DF000B0F1C04000F073B890EA010F0CEAD11363
:107E000048BF42F48072624538BF634504D280EABD
:107E1000010000F00040704710B500F01AF800BFF4
:107E20008900013E00F007B800F009B85FEA410C94
:107E30005FEA1C6C08D080EA010000F050B85FEAED
:107E4000400C5FEA1C6CF6D14FF00040A0F58000BA
:107E500070470EF1020E2EF0030E5EF8044B244222
:107E600004D44FEA4102B2F17F4F11D84FEA4003E8
:107E7000B3F17F4F0CD80ED14FEAD07CB2F17F4FD7
:107E80000CEB4C0C0CF1020C08BF4CEBD17C04E069
:107E90004FF0080C01E04FEAD17C0CEB4C0324FAC4
:107EA00003F404F00704B4F1040C06D20EEB840CC6
:107EB000BDE810404CF0010C6047DFE80CF007080B
:107EC00002024FF00040A0F5800010BD08464200BD
:107ED00018BFD2F1807288BF00F0004010BDFF21B2
:107EE00041EAD050C005704780F0004090EA010F91
:107EF0007FF56BAE81F0004100F007B890EA010F0A
:107F000048BF81F000413FF560AE421A04D882F0CC
:107F10000042A0EB020011444FEAD0524FF07F4CD8
:107F20001CEA410FA2EBD15318BF9CEA026F4AD062
:107F30004FF0004C4CEA00204CEA012121FA03FCEE
:107F4000B0EB0C0C0FD412F0FE0F36D05FEA4C00F1
:107F50001DD5001240EBC25038BF70471CF03F0FD8
:107F600018BF70470BE0A2F101025FEA1C2040EB52
:107F7000C25038BF70471CF07F0F18BF7047C3F165
:107F80002003994014BF401E20F001007047800874
:107F90004FEA122308BF7047B0FA80FCA2EB0C0234
:107FA000CCF1280C60FA0CF093EA122F04BF00EB1E
:107FB000C25070474FEAC3707047130A5FEADC1083
:107FC00008BF7047F6E79CEA026F04D010EA5C0F26
:107FD00008BF0020704710B5FFF73BFF40DFF63EBB
:107FE00081F0004070470CF00F03092B08BF0820F8
:107FF00000F059800A2B0BD0082B18BF704708BF20
:108000001CF0400F0AD04FF000004FF00001704705
:108010001CF0400F18BF4FF0004070471CF0100FCD
:1080200008D020F0704300F07F4242EAD3014FEACB
:108030004370704700F0604021F07F4242EA000246
:1080400001F07F4040EA727070474FF0FF0C4CF433
:10805000E06C1CEA11531CBF9CEA030C9445C2BFA0
:10806000DA4201EB02517047002B0DD0BCF1000F3A
:108070000FD0002A01F00041A4BF41F0E04141F0DF
:108080007F614FF00000704701F000414FF00000A9
:10809000704750EA01334FF09B0C18BF4CF0806CD6
:1080A0007FF4B2A970471CF4801F11D01CF4E02F9C
:1080B00003D06FEACC31490070474FF04050EFF3E6
:1080C000008222F0704242EA000282F30088704788
:1080D0004FF00000704700004C5555555555A53FD1
:1080E0007751C1166CC156BF9015CB19A001FA3E4D
:1080F000AD529C804F7E92BEC4B1B4BD9EEE213E77
:10810000D43888BEE9FAA8BD00004054FB21F93FED
:108110003163621A61B4D03D0000601A61B4D03D91
:108120007370032E8A19A33B0000002E8A19A33B0B
:10813000C14920259A837B3900000000000000001F
:108140006E83F9A22915444ED15727FCC0DD34F5C2
:10815000999562DB4190433CAB6351FE61C5BBDE48
:108160003A6E24B7E0D24D42EA2E49061C92D1095C
:108170001CEB1DFE3EA729B1F53582E88444BB2ED9
:1081800026709CE9417E5FB439D69139F439538326
:108190008B5F849C3B28F9BDFF97F81F0F9805DE85
:1081A0008B112FEF1F6D0A5ACF7E366DB709CB2783
:1081B000663F464F2DEA5F9EC7BA27757BF1E5EB18
:1081C000F739073DEA92528AB15FFB6B085D8D1F5C
:1081D000A6F810111111813FD561C119A0012ABF64
:1081E0007DFEB157E31DC73EEB9C2B8AE6E55ABEE8
:1081F0007CD5CF5A3AD9E53D288200000000001016
:1082000058010000000100005C82000000C007204F
:1082100034040000000100004883000034C407203B
:108220000C4F00005C010000910414E1F50576FF9D
:10823000FFFF7F010382A00F2DA8E4FFFF90290814
:1082400001108009F5285C3F0BD7A3C00524EB5132
:10825000B83E69E0410346E803000000110434E140
:10826000F5051EFCD10720AC041504D20720190423
:108270001AA00C1A20081A24041A28041A2C041A0A
:1082800030042A3420019B320C028F80320123DB20
:10829000381A99044B29390C23881323E8038B10CF
:1082A0002724092A5001C823FF031AF8041AEE04F0
:1082B0001AE1041AD0041ABA041A88041A6A041AB1
:1082C00049041A260411190423D8021AAF041A8586
:1082D000041A59041A2D0423F4011A7B041A5104B8
:1082E0001A280411190432DB32B732963278325D23
:1082F00032453230321F32127208290829102918EB
:108300002920292829302938294029482950295845
:108310002960296829702AD46C5984298C299429C8
:108320009C29A429AC29B429BC29C429CC29D42945
:10833000DC29E429EC29F429FC2380251AC08129B1
:088340000811224B02731B001F
:04000005000000C532
:00000001FF
